:10000000642D002009990000659900009197000077
:100010009197000091970000919700009197000040
:100020009197000091970000919700005D93000068
:10003000919700009197000019930000919700009C
:10004000CD98000017850000CD980000CD980000E5
:10005000CD980000CD980000CD980000CD9800000C
:10006000CD980000CD980000CD980000CD980000FC
:10007000CD980000CD980000CD980000CD980000EC
:10008000CD980000CD980000CD980000CD980000DC
:10009000CD980000CD980000CD980000CD980000CC
:1000A000CD980000CD980000CD980000CD980000BC
:1000B000CD980000CD980000CD980000CD980000AC
:1000C000CD980000CD980000CD980000CD9800009C
:1000D000CD980000CD980000CD98000000000000F1
:1000E0003512000000000000D59600009C0300209F
:1000F0000B0C000000000000D5960000000000007E
:10010000D596000000000000D5960000CC0300202A
:10011000B10F000000000000D596000000000000B4
:10012000D596000000000000D596000000000000F9
:10013000D596000000000000D984000000000000F7
:10014000D5960000000000001385000000000000AC
:10015000D596000000000000D596000000000000C9
:10016000D596000000000000510D000000000000C6
:10017000D596000000000000D596000000000000A9
:10018000D596000000000000D59600000000000099
:10019000D596000000000000D59600000000000089
:1001A0000D85000000000000D59600000000000052
:1001B000D596000000000000D59600000000000069
:1001C000D596000000000000D59600000000000059
:1001D000D596000000000000D59600000000000049
:1001E000D596000000000000D59600000000000039
:1001F000D596000000000000D59600000000000029
:10020000D596000000000000D59600000000000018
:10021000D596000053B94AB9002908BF00281CBF71
:100220004FF0FF314FF0FF3000F08EB9ADF1080C08
:100230006DE904CE00F01AF8DDF804E0DDE90223F0
:1002400004B07047430803F05533C01A830803F025
:10025000333300F03330184400EB101000F00F304F
:1002600000EB002000EB0040000E70472DE9F04746
:100270008C460D460446089E002B51D18A421746F3
:100280006DD9B2FA82FEBEF1000F0BD0CEF1200C78
:1002900001FA0EF520FA0CFC02FA0EF74CEA050CF6
:1002A00000FA0EF44FEA174A250CBCFBFAF81FFAC5
:1002B00087F90AFB18CC45EA0C4508FB09F3AB4269
:1002C0000AD9ED1908F1FF3280F02381AB4240F2E8
:1002D0002081A8F102083D44ED1AA4B2B5FBFAF062
:1002E0000AFB105544EA054400FB09F9A14509D968
:1002F000E41900F1FF3380F00A81A14540F2078143
:1003000002383C44A4EB090440EA08400021002ED6
:1003100061D024FA0EF4002334607360BDE8F087E6
:100320008B4207D9002E54D0002186E821000846D0
:10033000BDE8F087B3FA83F1002940F08E80AB422C
:1003400002D3824200F2FA80841A65EB0305012091
:10035000AC46002E3FD086E81010BDE8F08712B9F9
:100360000127B7FBF2F7B7FA87FEBEF1000F34D1D1
:10037000EB1B3A0C1FFA87FC0121B3FBF2F8250CAA
:1003800002FB183345EA03450CFB08F3AB4207D9DF
:10039000ED1908F1FF3002D2AB4200F2D180804665
:1003A000ED1AA3B2B5FBF2F002FB105543EA054487
:1003B0000CFB00FCA44507D9E41900F1FF3302D27D
:1003C000A44500F2B8801846A4EB0C0440EA0840AB
:1003D0009DE731463046BDE8F087CEF1200405FAAE
:1003E0000EF307FA0EF720FA04F83A0C25FA04F493
:1003F00048EA0308B4FBF2F14FEA184502FB114446
:100400001FFA87FC45EA044501FB0CF3AB4200FAF6
:100410000EF409D9ED1901F1FF3080F08A80AB426A
:1004200040F2878002393D44EB1A1FFA88F5B3FB8E
:10043000F2F002FB103345EA034500FB0CF3AB423C
:1004400007D9ED1900F1FF386FD2AB426DD90238F0
:100450003D44EB1A40EA01418FE7C1F1200722FA3F
:1004600007F88B4005FA01F448EA030320FA07FE77
:100470004FEA134CFD404EEA040EB5FBFCF94FEA7F
:100480001E440CFB19551FFA83F844EA054509FB85
:1004900008F4AC4202FA01F200FA01FA08D9ED18A8
:1004A00009F1FF3043D2AC4241D9A9F102091D4400
:1004B0002D1B1FFA8EFEB5FBFCF00CFB10554EEA0F
:1004C000054400FB08F8A04507D9E41800F1FF3502
:1004D00029D2A04527D902381C4440EA0940A4EBA0
:1004E0000804A0FB02894C45C6464D4615D312D0E0
:1004F00056B1BAEB0E0364EB050404FA07F7CB40E0
:100500001F43CC40376074600021BDE8F087184677
:10051000F8E69046E0E6C245EAD2B8EB020E69EB97
:1005200003050138E4E72846D7E7404691E78146CE
:10053000BEE7014678E702383C4445E7084608E74D
:10054000A8F102083D442BE7704700BFF8B5054607
:100550000E4601460848094F01F05EF90024AC42FE
:1005600001DB0020F8BD56F824202146384601F072
:1005700053F90134F3E700BFA3AC0000AEAC0000B8
:1005800008B5024801F048F9002008BDBFAC0000E2
:10059000704743685B68184743685B6A03B1184754
:1005A000704700000A2838B50446064D03D10D21D6
:1005B0002868FFF7EEFFE1B22868FFF7EAFF204660
:1005C00038BD00BF8004002000B5BFF35B8F50E84A
:1005D000003F43EA010240E8002EBEF1000FF6D1D1
:1005E000BFF35B8F18465DF804FB0000F8B5144EAE
:1005F00004460D4630680821FFF7CBFF37464DB95A
:1006000020213068FFF7C5FF30680821BDE8F840B9
:10061000FFF7BFBF0B4801F0FFF82544AC4208D1FB
:1006200038682021FFF7B5FF0748BDE8F84001F022
:10063000F3B8617804F8011B3868FFF7AAFFEDE70B
:1006400080040020EAAC0000EEAC00002DE9F04F81
:10065000DFF8E082AE4F85B0C146D8F800004368AD
:10066000DB6B1BB3984708B3D8F8000043689B6B5B
:10067000E3B19847D0B1D8F800004368DB6A002B9B
:10068000EBD098470028E8D0D8F8004063681B6991
:10069000002B00F06D8101220DF10F0120469847DB
:1006A000002880F265812046FFF776FF05B0BDE89F
:1006B000F08F082120460193FFF786FF019BCBF8BE
:1006C0000030944B00221A60C7E7BFF35B8F2368AA
:1006D000BFF35B8F1A0740F17D81A6F13003092B30
:1006E00017D8BFF35B8F2368BFF35B8F13F0100F36
:1006F0004FF00A0006D0874B1A6800FB0266303EB6
:100700001E60AAE784490B6800FB0366303E0E605A
:10071000A3E73B2E18D0BFF35B8F55E8003F23F0D3
:10072000080345E80032002AF7D1BFF35B8FBFF31F
:100730005B8F55E8003F23F0100345E80032002AA4
:10074000F7D1BFF35B8F45E110212846FFF73CFF4F
:10075000C306E0D481E7482E39D07E2E40F0458193
:100760006E4C2378002B00F0408101216C4801F091
:1007700053F86C4B217818780AF1040A0139C9B290
:1007800050442170FFF732FF2FE16648624A037838
:1007900011688B42C0F02981604ECCB232781B1BAD
:1007A000224403706048327001F036F81DE15B4866
:1007B000594B027819688A42C0F01781CBB2D21A1D
:1007C0000270584A1078034413705548ECE7554CB2
:1007D0002178002900F00981534801F01DF84F4AA3
:1007E000137821780B44137000232370FDE04B4CE9
:1007F0002178002900F0F980494801F00DF8494AB4
:10080000EEE7BFF35B8F54E8006F26F0010344E886
:100810000032002AF7D1BFF35B8F16F001069DF876
:100820000F500BD05B2D7FF418AF02212046FFF74D
:10083000CBFE04212046FFF7C7FE0EE7A5F12003FB
:100840005E2B4DD90D2D2DD015D8092D7FF405AF78
:10085000364B1B68002B3FF400AF304A1278002A59
:100860007FF4FBAE2F4C386821780430984723780A
:1008700018442070F1E61B2D12D07F2D7FF4EDAED1
:10088000284A1378002B3FF4E8AE013BDBB213702B
:100890003868224A043311781844FFF7A7FEDCE6D3
:1008A0000121C7E7DFF87CA01C4C9AF800103B68D8
:1008B0002278D9F800000B44134429461E71FFF733
:1008C00068FE0A21D9F80000FFF763FE184B39686B
:1008D00018688AF80060267009F02AFC3E60BCE6C1
:1008E0000E4A104B92F800B01E780BEB06027E2ADF
:1008F0003FF7B3AE3C68D9F80000721C29461A7065
:10090000FFF747FEA319BBF1000F15D11D71A4E637
:100910006C040020640400206004002075040020A2
:1009200026AD00007404002020AD000070040020FB
:100930007C0400208004002093F804A031481D713D
:10094000043600F069FF34440BF1010B661C5C4473
:10095000B44203D12C4800F05FFF7EE65146D9F83F
:100960000000FFF716FE337806F801AB9A46EFE772
:10097000396839B9254B186809F028FC3860002817
:100980003FF494AEBFF35B8F214C2368BFF35B8FC2
:1009900013F0020F25463FF434AF9DF80F60D7F8EF
:1009A00000A0BFF35B8F55E8003F23F0040245E849
:1009B00000210029F7D1BFF35B8F59077FF585AE82
:1009C000A6F13003092BDFF84CB07FF672AE01239D
:1009D000CBF80030462E3FF40AAF3FF6BCAE432EB4
:1009E0003FF4E5AE442E3FF4D0AEBFF35B8F55E845
:1009F000003F23F0020345E80032002AF7D1BFF39D
:100A00005B8F2AE6EAAC0000EEAC00006804002030
:100A10007804002060040020174B13B51860174BB2
:100A2000174C1960174B20681A60FFF7B5FD206856
:100A300043689B6903B19847206843681BB11B6CEE
:100A40000BB11149984720684368DB6A2BB92068CD
:100A500043681B6A73B902B010BD98470028F6D0EE
:100A6000206843681B69002BEDD001220DF10701BE
:100A70009847E8E79847EEE7680400207C040020E8
:100A800080040020700400204D060000014800F0A2
:100A900093BD00BFA505000008B5044808F0B0FFED
:100AA000034B1860FFF7F2FF002008BDF2AC000016
:100AB0008004002003689B681B68D3F8082132B1CA
:100AC0000020C3F80801D3F818350B7070474FF0B9
:100AD000FF30704703689B681B68C3F81C15D3F888
:100AE0001C21002AFBD00022C3F81C2108467047B5
:100AF00003689B681B68D3F8240118B1D3F88004FD
:100B0000C3F8800400F00F00704770B503689B685D
:100B10001C6800231E46D8B2151A002D03DDD4F838
:100B20001C51013305B970BDC4F81C61085CC4F8E0
:100B30001C05F0E770B503689B681C6800231E461F
:100B4000D8B2151A002D03DDD4F80851013305B9C8
:100B500070BDC4F80861D4F818550D54F0E7036867
:100B60009B681A68D2F8043343F00803C2F80433D0
:100B7000704703689B681A68D2F8083343F008038B
:100B8000C2F80833704703689B681B68D3F81C01E0
:100B9000704703689B681A68D2F8043343F0040373
:100BA000C2F80433704703689B681A68D2F80833A8
:100BB00043F00403C2F80833704703689B681B685E
:100BC000D3F81C01B0FA80F04009704703689B68B5
:100BD0001B68D3F80801704703689B681A68D2F84D
:100BE000043343F01003C2F80433704703689B6872
:100BF0001A68D2F8083343F01003C2F8083370477C
:100C00000120704783685960704783685B6803B14F
:100C10001847704708B502200022012108F042FD64
:100C20000220BDE8084008F013BD08B50246FFF7F2
:100C3000AAFF30B91046FFF7C9FF003018BF0120E6
:100C400008BD012008BD0000F8B503689B68054693
:100C50001A481C6808F0D4FE436806461F680D2237
:100C600040F201130021B84773681F68002319463A
:100C70000F223046B8470D23C4F80C350F23C4F8B3
:100C80001435AB684FF4E1321A602B689B681A6820
:100C90009B684FF0EB71C2F824150422C4F80025BC
:100CA00000260122C4F81C61C4F80861A260226019
:100CB000034A6A60284698473046F8BD03AD0000F5
:100CC00038AD0000084BC3F84005D3F80435C01A0E
:100CD00020F07F40054B0238984282BF044B4FF40E
:100CE0000032C3F80021704700100140FDFF7F0073
:100CF00000E100E010B5124B124CD3F80405226855
:100D0000801A20F07F40B0F5A37F11D90E49096801
:100D100040F24713B0FBF3F0884228BF084603FBBC
:100D2000002323F07F432360084B186009F0DCFCAC
:100D30002068BDE8104000F24710FFF7C3BF00BFB6
:100D40000010014088040020840400205803002083
:100D5000024B0022C3F84021FFF7CCBF0010014036
:100D600046F23543984228BF1846054B1860054B9C
:100D70001B6840F2471202FB0030FFF7A3BF00BF21
:100D8000840400208804002008B5074B0022C3F823
:100D90004021064B4FF40032C3F88021FFF7AAFF31
:100DA000034B01221A6008BD0010014000E100E081
:100DB0008404002070B5184808F022FE48B3436848
:100DC000164D1B6801219847154B00241C60154BDC
:100DD00001261E6040F24713C5F80845C5F84035A6
:100DE0004FF48033C5F84433C5F804330E4BC5F8CF
:100DF00040414FF40032C3F8802131462246112091
:100E000008F050FC112008F023FCAE6020462E6054
:100E100070BD4FF0FF3070BD0AAD00000010014002
:100E2000880400208404002000E100E030B50B4A73
:100E30000B48D2F80415D0E90045D2F804359942A0
:100E40000AD1084A40F2471303FB1413106823F039
:100E50007F4300FB043030BD1946ECE70010014031
:100E6000C81600205C03002003689B689A688368AA
:100E700010B5DC68002024FA00F3DB0707D500F585
:100E8000A27352F82330C3F304238B4204D0013001
:100E90000828F0D16FF0120010BD0068806800686B
:100EA00041B9D0F8101521FA02F202F001021A60DD
:100EB00000207047D0F81025F9E7006880680068C6
:100EC00049B9012191401BB1C0F8081500207047B5
:100ED000C0F80C15FAE7C0F80435F7E710B58368D9
:100EE0003AB11A680A605A68196002B9596000205C
:100EF00010BD18680028FAD081420ED15C680868DD
:100F000032B9A142186000D1586000230B60EEE7AF
:100F1000A142106008BF5A60F7E702460068E9E79F
:100F2000F8B514460268876892680D469668A1B9BC
:100F30002146FFF799FF002811DBBA68012303FA65
:100F400004F4144300F1400203FA00F0BC6046F8D8
:100F50002250C6F804032846F8BD6FF02200F8BD01
:100F6000F8B514460268866892680D46976889B994
:100F70002146FFF779FF00280EDBB268012303FA50
:100F800004F403FA00F022EA0404B460C7F808038A
:100F90002846F8BD6FF02200F8BD08B500220121F7
:100FA000062008F07FFB062008F052FB002008BD59
:100FB000F8B5036806469B68B46898680022134633
:100FC0001546012700EB8201D1F800E1BEF1000FC8
:100FD00008D0C1F80051D1F81015C1F3042107FA67
:100FE00001F10B430132082AECD1A56806201D400F
:100FF00008F03CFB246824B90620BDE8F84008F05E
:1010000027BBA3681D42F5D063682A4621463046B7
:101010009847EFE72DE9F84314460268876892681D
:1010200080469568166819B16FF02200BDE8F88314
:1010300003F44071B1F5807FC3F30132C3F381390A
:101040004FD0B1F5007F0CBF0420002013F0010F3A
:10105000DFF8B8C04FEA820204F5E07E4AD00C28DF
:1010600041D10121A140C6F808154A445CF822206C
:1010700042F00302024313F0020046F82E2043D050
:101080009906D1D55A063AD413F0040F14BF4FF481
:1010900080364FF40036F868FFF7D4F8082831D0CE
:1010A00021464046FFF7E0FE0028FB6808DADA43F5
:1010B00092FAA2F0002AB0FA80F008BF4FF0FF3099
:1010C0002402012204F4F854824044F0010400F5A3
:1010D000A27013433443FB6045F820400020BDE874
:1010E000F8830C20B2E7042802BF0121A140C6F812
:1010F0000C15BAE702EB09015CF82120BAE74FF4BE
:101100004036C8E76FF00400BDE8F8837CAD00000E
:1011100010B54FF02003EFF3118283F31188114CC7
:10112000237823B982F311886FF0440010BD013B8E
:10113000DBB223701BB182F31188002010BD0A4B73
:101140001878012128B1217082F311886FF00A000C
:1011500010BD197082F311884FF0804251601870F1
:1011600010BD00BF9D0400209C04002008B5002293
:101170001046012108F096FA002008F069FA0020D4
:1011800008BD0000F8B54FF02002EFF3118382F3A1
:101190001188254A1078441C147060B183F31188BB
:1011A0004FF08043D3F80C3413F4803F14BF002079
:1011B0006FF04300F8BD1D4D2F782FB1107083F3F1
:1011C00011886FF00A00F8BD01262E7083F3118894
:1011D0004FF0804419B3384608F048FAC4F800715B
:1011E000D4F80433C4F804632660D4F8002192B123
:1011F0000022C4F800210E4A13F0010F4FF0010342
:1012000008BFC4F808330020C2F8803108F020FA83
:1012100000232B70C4E720BF40BF20BFE5E7C4F820
:1012200000112660F4E700BF9D0400209C0400200C
:1012300000E100E0F8B54FF080430546D3F808E13F
:10124000D3F80423D3F80C44D3F80071D3F8040185
:10125000D3F80C11D3F8106102F00102BEF1000FB7
:1012600003D04FF0000EC3F808E127B14FF08043E0
:101270000027C3F800713AB1E30341BF4FF0804348
:101280000122C3F808231A6120B14FF080430022E5
:10129000C3F8042149B14FF080440021C4F80C1177
:1012A0002846FFF735FF0123636176B14FF0804395
:1012B00000210124C3F810112846C3F80443FFF7A6
:1012C00061FF10B9014BC3F80041F8BD00E100E037
:1012D000F8B54FF080440746D4F8186416F4803609
:1012E0000D4648D1304608F0C1F9C4F80461022225
:1012F000D4F80433C4F804230122C4F81855A260BA
:10130000D4F804219AB39B0758BF02234FF0000280
:101310001A4EC4F8042158BFC4F808330124C6F893
:101320008041002008F094F94FF0804300211822FA
:10133000C3F80823C3F80C11C3F8101115F003010A
:101340000CD11020C3F83805C3F804233846C3F87D
:101350000443FFF717FF08B9C6F800414FF0804378
:10136000D3F8180480F48030C0F30040F8BD20BFEB
:1013700040BF20BFC4E70020F8BD00BF00E100E08F
:101380004FF0847070470139034611F8012F0AB9F4
:101390001A70704703F8012BF7E710B501390346BF
:1013A0003AB111F8014F2CB91A4403F8014B93429A
:1013B000FBD110BD03F8014B013AF1E7C9B2034676
:1013C00010F8012B914206D0002AF8D100290CBF59
:1013D0001846002070471846704702460346981A80
:1013E00013F8011B0029FAD170470138013910F8B0
:1013F000013F11F8012F934202D1002BF7D11A4679
:10140000981A704710B501390244904209D0037808
:1014100011F8014FA34200D10BB9181B10BD0130C8
:10142000F3E7002010BD38B504460D46FFF7D5FFA1
:1014300029462044FFF7A7FF204638BD70B582B18A
:10144000013A0C46034603D11A782078101A70BD71
:101450001E782578AE4200F1010001F10101EFD0C4
:10146000F2E7104670BD81EA000313F0030F70B578
:1014700003460BD0013B0A4491421BD170BD002AA8
:10148000FCD011F8014B03F8014B013A9C07F6D14F
:101490001E1F0D46541B0C44032C06D822F00304D7
:1014A0002144234402F00302E4E755F8044B46F8D4
:1014B000044FEFE711F8014B03F8014FDCE770B57B
:1014C000C9B203469C0711D141EA012444EA04440D
:1014D0001E46951B1D44032D0ED822F00304234401
:1014E00002F003021A44934209D170BD002AFCD0D5
:1014F00003F8011B013AE5E746F8044BE9E703F876
:10150000011BF0E7002070470B6801330B60014BB3
:101510001B6818472C0000202DE9F04F85B09B4632
:101520000E9CDFF890A0012CB8BF0124012B0CBF4A
:1015300030232023154680468946019402930126D4
:101540000A2700220AF101040AB9AA451FD2B5FBF5
:10155000F4F049463030C04701360122013F012FE7
:10156000B5FBF4F14FF00A0304FB1155BAFBF3FA93
:10157000E8D1494605F13000C047BBF1030F03D164
:10158000019B9C1B002C0FDC05B0BDE8F08F019B7C
:10159000BB42E3DBBBF1020FE0D84946029803925D
:1015A0000136C047039AD9E749462020C047013C8D
:1015B000E8E700BFFFC99A3B014B1860704700BFC6
:1015C0002C0000202DE9F04F89B04FF0000A0646AC
:1015D0000F4604921C464FF0FF39D0465546049BF7
:1015E000187810B909B0BDE8F08F45B9252800F08A
:1015F000F8803946B047049B01330493EFE7642831
:1016000055D018D839280AD8312844D22D2830D0BE
:10161000302831D0252807D13946B04763E0582813
:101620007DD0632800F0D78039462520B047049B41
:1016300039461878F1E7702867D006D8692836D07F
:101640006C2831D06828D6D0EEE775284DD00CD85C
:101650007328E9D104F1040B2468013C14F8010F4C
:10166000002840F0B5805C463DE0782857D07A28C5
:10167000E9E74FF00308BEE7B9F1000F0EDAB8F161
:10168000000F00F0B480A0F13009B8F1000F08BFDE
:101690004FF00208AFE7B9F1000FF4DB0A2303FBB8
:1016A0000909A9F13009F0E70AF1010AA3E7BAF143
:1016B000010FC5BF073424F0070325681D68D4BF98
:1016C000043403F10804002D05DA39462D20B04713
:1016D0006D4209F1FF39CDF8009043462A4639465C
:1016E0003046FFF719FF002585E7BAF1010FC5BFA6
:1016F000073424F0070322681A68CDF80090CCBFA5
:1017000003F1080404344346E9E739463020B04782
:1017100039467820B0474FF008094FF00108BAF178
:10172000010FC7BF073424F0070323680593C2BF26
:1017300003F108041B6805934FF008024FF0000303
:10174000D8BF04340393079393460BF1FF3B059BEB
:101750004FEA8B0023FA00F010F00F0009D1079B2D
:1017600013B9BBF1000F22D14FF0300E07E0069AFB
:10177000EBE709288CBF4FF0570E4FF0300E39467B
:1017800070440692B047039B079501330393BBF166
:10179000000FECD1B8F1030F2CD1039BC3EB49052B
:1017A000002DA0DD39462020B047013DF8E7531E4B
:1017B00091450693EBDBB8F1010F03D13946302098
:1017C000B047E4E7B8F1020FE1D139462020F7E74E
:1017D0003946B04742E72068251D3946B0472C46B8
:1017E00081E7AA46A8464FF0FF39012503E74FF0ED
:1017F000010800E75D46FEE613B502AC002344F89D
:10180000043D02460B4603482146FFF7DBFE0198E4
:1018100002B010BD091500000FB407B504A951F8B6
:10182000040B0191FFF7E8FF03B05DF804EB04B08F
:1018300070477047438A1844173020F00300704700
:1018400000B5BFF35B8F50E8003F43EA010240E878
:10185000002EBEF1000FF6D1BFF35B8F18465DF886
:1018600004FB00B5BFF35B8F50E8003F03EA0102C1
:1018700040E8002EBEF1000FF6D1BFF35B8F184693
:101880005DF804FB08B502460846FFF7D3FF43683E
:1018900043B142700846FFF7CDFFBDE808404068FD
:1018A00008F0B6BE08BD0000074BBFF35B8F4209CE
:1018B00003EB820300F01F00DB6EBFF35B8F43FA84
:1018C00000F000F00100704730000020F8B5054638
:1018D0000E460F484FF0FF3107F05AF8002104463A
:1018E00007F091F82046FFF7A5FF0022027020467E
:1018F000FFF7A0FF45802046FFF79CFF03214260D1
:1019000004F10C0007F0ABF8867005802046F8BDA6
:101910000001002030B5154687B00C4619B9FFF715
:10192000D5FF044648B301220021684608F05AFE5C
:101930002046FFF77FFFC0F804D0204607F08BF861
:1019400021460F4807F064F842F21071684608F02B
:10195000A3FE2046FFF76EFF407830B1204607F027
:1019600064F86FF0040007B030BD0DB12C60FAE7E9
:10197000204607F05AF82846F5E76FF03600F2E700
:10198000E400002070B5154D062205F10801064659
:10199000FFF754FD0446D8B1062142F20500FFF7D7
:1019A00095FF0446B0B1062231460C3007F05DF8D1
:1019B0002146002242F20500FFF7ACFF044638B989
:1019C0000622314605F10800FFF74DFD0123EB71BA
:1019D000204670BD6FF03604FAE700BF30000020EB
:1019E00037B50720FFF760FF70B3022142F20C0009
:1019F000FFF76CFF044650B302210C3007F02FF8BC
:101A0000022205460021FFF75AFD002321466B7094
:101A10002B7001AA42F20C00FFF77CFF044680B94C
:101A2000019BDB681C784CB96FF080010948FFF717
:101A300018FF6FF400710748FFF713FF019806F0D5
:101A4000F4FF204603B030BD6FF04404F9E76FF0B7
:101A50003604F6E79C00002008B50820FFF724FFB5
:101A600038B90720FFF720FF18B1BDE80840FFF79D
:101A7000B7BF002008BD012310B50621044600F8B9
:101A8000013B02F015FC18B9A37963F03F03A37181
:101A900010BD00007FB5002102AA40F60340FFF709
:101AA00039FF0446002840F03081029BDB681B7838
:101AB0006BB9C14A1360C14BBFF35B8F012253E87E
:101AC000001F43E800200028F9D1BFF35B8F029884
:101AD00006F0ABFF02AA002141F20300FFF71AFF54
:101AE0000446002840F01181029BB54DD9680822B8
:101AF000013105F11600FFF7B6FC029806F095FFDC
:101B0000214602AA41F20100FFF704FF0446002823
:101B100040F0FB800298C3685A78AA73D9789A7803
:101B200042EA01222A821A79EA73197ADA7942EAB8
:101B300001226A825A799B7942EA0323AB8206F03A
:101B400074FF214602AA41F20900FFF7E3FE0446B2
:101B5000002840F0DA80029BD96806220131681C17
:101B6000FFF781FC02982C7006F05FFF214602AA65
:101B700041F20200FFF7CEFE0446002840F0C58087
:101B8000029BD9684022013105F11E00FFF76BFC72
:101B9000029806F04AFFAB7E580640F10A812146C2
:101BA00002AA42F20300FFF7B5FE0446002840F007
:101BB000AC80029BD9680822013105F17000FFF763
:101BC00052FC029806F031FFAB7E990640F182800C
:101BD00095F83A301A0700F19B80082142F2010083
:101BE000FFF774FE044600287BD008210C3006F075
:101BF00036FF95F8403003F00603062B14BF02238E
:101C00004FF4C173002203701B0A43708270C270CC
:101C1000027142718271C271214642F20100FFF7E6
:101C200079FE0446002870D1082140F60140FFF7F4
:101C30004DFE0646002854D008210C3006F00FFF58
:101C4000802343700223C3702023047084700471C6
:101C500044718471C3712246314640F60140FFF75A
:101C600059FE0446002850D100900722CDF8030009
:101C700069465348FFF7E2FB00285CD1514E3368B8
:101C8000002B69D14FF08053D3F8A420013206D144
:101C9000D3F8A8304FF6FF729BB2934277D04FF043
:101CA0008052D2F8A030DB0771D501232B70D2F817
:101CB000A4306B70C3F307211B0CEB701B0AA970D7
:101CC0002B71D2F8A8306B71C3F3072363F03F0385
:101CD000AB7149E0022140F66D40FFF7F7FD064683
:101CE00010B96FF0360410E002210C3006F0B7FE98
:101CF0000123447003702246314640F66D40FFF7E1
:101D000009FE044600283FF463AF204604B070BDCE
:101D100002AA002142F21C00FFF7FCFD0446002845
:101D2000F3D10298C36853F8012F5B68EB67AA6789
:101D300006F07BFE51E7244B18689A8802909B7945
:101D4000ADF80C2002A907221D488DF80E30FFF7D0
:101D500075FB002892D0D8E700211C68184A072399
:101D60000846A04707288DD12B78012B1ED1AB79CF
:101D700003F0C003C02B19D11448FFF703FE04463B
:101D80000028C2D104210D48FFF75AFDBDE70C48D9
:101D9000FFF771FE04460028B7D13368002BE3D06B
:101DA0005E68074A07230146B047DDE76FF0150478
:101DB000ABE76FF01204A8E7EC0400209C000020C1
:101DC00030000020CC1500208CAC00003100002039
:101DD000064B4FF0FF3041F6FF71C3E90001044BA1
:101DE0001F200021C3E90001704700BF50010020FF
:101DF0005801002010B5FFF74DFE044630B902210E
:101E00000648FFF71DFD2046FFF726FE044B1B6822
:101E10001BB12046BDE81040184710BD9C000020B3
:101E2000E80400208368DB8B032B2DE9F74F044681
:101E300004D806F0FAFD6FF0150028E0FFF7FAFC71
:101E40000678012E3DD1E7683B780E3B012B3AD84E
:101E5000404080F311884FF0040002DFE6684048FC
:101E60006FF01001FFF7FDFC337843B9711C40227D
:101E70003C48FFF7F8FA39463948FFF7E1FC3A4B9E
:101E80001D68771C35B9204606F0CFFD002003B051
:101E9000BDE8F08F32782B68002A0CBF384600204E
:101EA00098476D68EEE7314DE0682A68002AEAD06D
:101EB000037823B90130904700232B60E3E700202B
:101EC000F9E72046B5E704F10C050221284606F0A3
:101ED000D5FD3B783E2BD6D1E7683146284606F043
:101EE000CDFD3F78082FB9D0092FDCD0022FCAD101
:101EF000284606F0CBFD1E4F009004F1140A009B0B
:101F0000002BC0D009212846D4F80C8006F0B6FD7D
:101F10003B68D3B198F8083043442846597A019178
:101F200006F0BCFD98F808300199B4F810B023828F
:101F3000814640462B4610F8012B3E6849B2B04717
:101F40001AFA89F3E360A4F810B098F8081028464C
:101F5000013106F093FD009B5E1EF3B20093CEE7C5
:101F60009C000020A4040020E4040020A004002021
:101F7000EC0400202DE9F0410446C668FFF75AFC46
:101F80000378012B05D0404080F311884FF0040006
:101F900002DF238A012BF6D933780E3B012BF2D8CE
:101FA00004F10C050221284606F068FD3378194E2D
:101FB0000E2B05D00F2B1BD0204606F036FDE2E796
:101FC000E368032128461F7806F058FDA368B34252
:101FD00004D1E36821461878FFF754FC17B10E4886
:101FE00008F016FB204606F020FD0020BDE8F08139
:101FF000E7680421284697F8018006F03FFDA368B2
:10200000B34203D121463878FFF73CFCB8F1000F0A
:10201000E8D0E4E700010020B0000020084AD2F830
:10202000CC303BB9816841B1C16831B1C2F8CC0054
:10203000184670476FF0440070476FF01500704706
:102040003000002038B50546064806F0A1FC0446DD
:1020500030B1002106F0D7FC2046FFF7EBFB0570FE
:10206000204638BD2801002010B501464FF020035E
:10207000EFF3118083F311880C4B0022D3F89840C2
:10208000C3F8982080F3118824B90120BDE81040DE
:10209000FFF7D8BF2046FFF7CDFB012303701146A1
:1020A0002046228206F0AFFC204610BD3000002002
:1020B00038B50C300D460221144606F0D0FC0570F0
:1020C000447038BD38B505464FF0FF30FFF7CCFF00
:1020D000042204460F21FFF7EBFF042104F10C005A
:1020E00006F0BDFC01234370024B05701B88438042
:1020F000204638BDF004002038B504464FF0FF30CC
:102100000D46FFF7B1FFEA1C2060D2B20E21FFF7A7
:10211000CFFF206803210C3006F0A1FC01230370DF
:10212000054B1B88A0F80130206829460C30BDE81B
:10213000384006F094BC00BFF004002070B504469F
:10214000154601320E460C34D2B23E21FFF7B0FFE5
:102150000121204606F083FC067029462046BDE892
:10216000704006F07CBC00000E4B70B51546D3E9FC
:102170000023002302F08002134304460E4610D0D1
:10218000042208212846FFF793FF042105F10C00E3
:1021900006F065FCB4FA84F35B090470A0F80160F2
:1021A000C37070BD5001002070B504461846134B33
:1021B0001646D3E90023002203F0005313430D46D3
:1021C0001BD00F4BD3E90023002302F00802134376
:1021D00013D00B220421FFF7B1FF08220470A0F8EE
:1021E0000160033024B9291DBDE87040FFF73BB9F9
:1021F0000021BDE87040FFF762B970BD50010020BA
:1022000058010020034600685968704730B5018ABC
:102210008BB0002302290446059302D800200BB09E
:1022200030BDC368C34D1A7858789B7842EA0022C3
:102230008B422A80F2D8032104F10C0006F01EFC28
:102240002B88DAB29B0A013B072B09D8DFE803F0A1
:1022500004082140080808A2062A07D01D2A13D026
:10226000012105A8FFF748FF012314E1E3689978ED
:10227000188806F029F8002814BF0C200020FFF76A
:1022800021FF05900598CAE7E368188806F008F86A
:10229000F1E7012A15D0032AE2D1A74B4FF0FF3016
:1022A00041F6FF71C3E90001A44B1F200021C3E9DF
:1022B000000105F0EDFD012105A8FFF71DFF00233A
:1022C000E9E0E068FFF79EFF9B4BC3E90001F2E7FE
:1022D000013A082AC4D801A353F822F001230000D0
:1022E000252300006123000061220000612200001C
:1022F0006122000061220000612200007D230000B5
:10230000092105A8FFF7F8FE002309220370837056
:10231000C3704FF0FF334270027143718371C37118
:102320000372AFE7412105A8FFF7E6FE002104464E
:10233000402200F8011BFFF7C2F820236370C0237E
:10234000A3712823E37302232374F723A376FF23C7
:10235000E37623770F236377302384F8223091E7E5
:10236000092105A8FFF7C8FE00210446082200F84D
:10237000011BFFF7A4F86023637183E7072105A819
:10238000FFF7BAFE0146002301F8013B184606F0AC
:1023900091F977E7013A1B2A3FF662AF01A353F8A0
:1023A00022F000BF152400001F2400003724000085
:1023B000612200005924000017250000412500007B
:1023C0004F2500005B25000067250000612200000A
:1023D00061220000612200006122000063240000ED
:1023E000752400007B2400009B2400006122000073
:1023F000612200006122000061220000B924000077
:10240000DF24000061220000612200006122000040
:10241000F5240000E068FFF7F5FE484B55E704217E
:1024200005A8FFF769FE002303701B2283700223B7
:102430004270C37026E7092105A8FFF75DFE00255D
:102440000446082200F8015B2946FFF738F80F23FD
:102450006370A570E57015E7E168012006F042F9A8
:1024600029E7022105A8FFF747FE00230370082390
:10247000437007E705F054FD1DE7E368591C187821
:1024800005F056FD0121044605A8FFF735FE002C96
:102490000CBF002307230370F4E6E368591C187887
:1024A00005F06AFD0446012105A8FFF725FE002C72
:1024B0000CBF00230C23EEE7E06806AA002300F11E
:1024C000100100F0C3FC112105A8FFF715FE002341
:1024D00000F8013B102206A9FEF7C5FFD2E609214C
:1024E00005A8FFF709FE002300F8013B082101F0D1
:1024F000DFFEC7E6092105A8FFF7FEFDFF23002246
:1025000043708370C370037143710323027083713E
:10251000C2710272B6E6E468A57BA379627921797B
:1025200020880295657B01950734009406F0E6F853
:10253000C1E600BFF0040020500100205801002037
:10254000022105A8FFF7D8FD0023037090E7E36898
:10255000591C187806F05CF9ADE6E368591C187848
:1025600006F0A4F9A7E6E368187806F0DBF999E726
:102570000379012BF7B504460E465AD0022B40F0E2
:102580000F8101228DF801208DF806300322874B40
:102590008DF80220FF228DF803208DF80520D3E965
:1025A0000023002203F000530025042113438DF87B
:1025B00000508DF804103AD07D4BD3E9002300235E
:1025C00002F00202134332D0037A03F00F03012B0F
:1025D0001EBF457A063DEDB205F10B02D2B20221D3
:1025E0003046FFF7ABFD01230370237A02AA03F004
:1025F0000F031344274613F8083C437017F8083FAD
:102600000646C3F38013837004F10A0106220330E7
:10261000FEF729FF0A3606F8015C2A4607F1080191
:102620003046FEF720FF637A1C44A37A735503B04B
:10263000F0BDC37AC588033B122B00F2B180DFE8FE
:1026400003F00AAFAF31A6AF39AFAF4362AF66AFA9
:10265000AFAFAF868600554BD3E90023002203F0CD
:1026600000531343E3D0524BD3E90023002302F07D
:1026700010021343DBD00C2205213046FFF75EFD2C
:1026800004F10C010646082220F8025BFEF7EBFE7F
:10269000022204F1140106F10A0003B0BDE8F04083
:1026A000FEF7E1BE0A460020294603B0BDE8F0402F
:1026B000FFF75ABD0B462A4600F10801002003B07F
:1026C000BDE8F040FFF770BD384BD3E9002300238D
:1026D00002F400621343AAD007220C213046FFF710
:1026E000E7FC072106F10C0006F0B9F9002303709E
:1026F000A0F80150237BC370B4F80D308380B4F888
:102700000F30837193E70A46007B2946CDE7274BBC
:10271000D3E90023002203F00053134387D0244B56
:10272000D3E90023002302F0200213433FF47FAFDC
:102730000A2206213046FFF701FD0580A389438068
:10274000E3898380238AC380638A03816FE7174B01
:10275000D3E90023002203F0005313433FF467AF93
:10276000134BD3E90023002302F0400213433FF44C
:102770005EAF0A2207213046FFF7E0FC0580238A7E
:102780004380638A8380A389C380E389DDE7037B79
:102790000E2B7FF44CAF0B462A4600211A208EE701
:1027A000404080F311884FF0040002DF5001002008
:1027B000580100200379012B06D0023BDBB2042B29
:1027C0000AD8074AD0567047037A03F00303032B55
:1027D0000CBF0220032070474FF0FF30704700BF4E
:1027E000FCAD000008B50248FFF718FC002008BD4A
:1027F00004AE000010B5038A044683B1438A034443
:10280000173323F003031B784BB9FFF7FFFC08B124
:10281000FFF7B0FB204606F008F9002010BD6FF06E
:10282000150010BD1FB500239A4202D0CC5CAA2C23
:102830000DD0D41A642161430192B1FBF2F10094EE
:10284000029101460348FEF7E7FF04B010BD0133D3
:10285000EAE700BF2BAE000073B5254E254D4FF0C3
:10286000FF31304607F0B2FC044620B3FFF7A2FF69
:102870000228019433D801280EBF00214FF0FF3108
:102880000120FFF7DFFB044618B101460198FFF76E
:102890006FFE019B0021D88805F0F2FD02A80022FE
:1028A00050F8043D1A6005F08DFD24B1238A2046BE
:1028B000DBB1FFF7B7FA07F0DFFD07F00BFF2B687E
:1028C000C01A41F288339842C9D94FF480620A494C
:1028D0000A48FFF7A7FF07F0FDFE2860BFE740406A
:1028E00080F311884FF0040002DF06F09EF8E2E763
:1028F00048040020F80400203824002019AE00000D
:1029000073B5154E154C164D0DF1020101A805F0D9
:10291000EFFC0028F8D1019B33B105F021FD0199AE
:10292000104807F005FCEFE74FF0FF31304607F0A5
:10293000B3FE07F0CFFE2368C01A41F288339842F5
:10294000E2D94FF4E07229460748FFF76BFF07F022
:10295000C1FE2060D8E700BF18040020F404002066
:10296000D81900204804002014AE000010B5144807
:1029700086B005F029FE0446F8B9FFF729FA6FF092
:10298000090303934FF4E0720E4B0F49059404942E
:102990000294019400940D4808F04EF86FF008037B
:1029A000039305940494029401940094084B0949FC
:1029B00009484FF4806208F03FF8204606B010BD89
:1029C0001804002001290000D8190020401600201A
:1029D0005928000038240020D01500202DE9F047A8
:1029E000114FDFF848900426013EF6B2FF2E19D0B1
:1029F00033B24FEA830803EB43031D0104244FF075
:102A00000C0A0AE01AFB04510A1D04EB08003A44C0
:102A1000394409EBC00000F080F9013CE4B2FF2C1E
:102A2000F0D1E1E7BDE8F0877C050020FC04002040
:102A3000F0B4124B05460F460C26302472B16143A8
:102A400006FB00142344597A187A814204BF0131ED
:102A5000197228463946F0BC05F06CBD4C4306FBA4
:102A6000004423449C7ADA7AA24204D101329A7259
:102A7000F0BC05F08DBDF0BC704700BF7C050020A8
:102A8000F8B505460E461C468AB1012362782078C7
:102A9000801A10F0030729D003B3012F39D0013277
:102AA000D2B222703146284605F072FD1CE005F0D6
:102AB0005DFD0028E9D03146284605F049FD002893
:102AC000E3D030230C22734302FB0533124A1A442D
:102AD000937AD27A9B1A18BF0123D7E70232D2B277
:102AE0002270E368A06898470020F8BD002BF8D05A
:102AF0000132D2B222700423302212FB06320C23A0
:102B000013FB0523044A61681A44204600F008F9C3
:102B1000C8E73846F8BD00BF7C0500202DE9F04F1E
:102B200000EB400389B01B014FF00008434E0493B3
:102B300005460424CDF80480013CE4B2FF2C0BD1FF
:102B4000019B002B76D0B8F1000F73D14246294685
:102B5000284605F0EFFC6DE00DF1200B00230C275B
:102B60004BF8043D4FF0300907FB04F309FB053136
:102B700070185A4671584068029300F0D8F8049BC8
:102B800017FB0437F31982460393BAF1000F19D1EA
:102B900030220C236A4303FB04223244917AD07A18
:102BA00088421EBFD1720122019230226A4303FB88
:102BB000042333441A7A597A91421CBF5A724FF057
:102BC0000108B9E7079B1F785A78BF1A07F0030777
:102BD000012F04D1013A5A709868DA689047079A31
:102BE00013785278DBB29A1A02F00302012A059395
:102BF0000DD0029B039909FB053030440022406848
:102C000000F09EF8079A059BC2F804A05370029B3F
:102C100009FB0533F0185A46F158406800F087F870
:102C2000012F8246B1D10CB90028B1D029462846DF
:102C300005F0AEFC09B0BDE8F08F00BF7C050020B8
:102C4000F7B51860C31D054623F00303501E0E465A
:102C500080B214461A800021042206FB0050FEF7C1
:102C60002EFC023CA4B24FF6FF77BC4201D103B068
:102C7000F0BD04FB06602B180422801B0DEB020143
:102C80002844013C0193A4B2FEF7EDFBEDE773B5D8
:102C90000568064695B1EB1D23F0030304221C884A
:102CA00029460DEB0200FEF7DEFB019B013CA4B2BE
:102CB0001BB1DA1D22F0030214803360284602B0F3
:102CC00070BD70B50C6806460D461CB1E31D23F0BF
:102CD00003031C88042229463046FEF7C4FBF21D7C
:102CE00022F00302631C13802E6070BD02FB010002
:102CF0007047401A80B2B0FBF2F0704710B5114433
:102D000001384FF6FF73013A92B29A4200D110BDDA
:102D100011F8014D00F8014FF5E7106008607047A9
:102D20001368196013685860116008467047814243
:102D300004D00AB14B681360084670470021FBE7D6
:102D40000B68834206D00AB1586810601A680A609E
:102D50001846704700231B68FFDE10B5421E002096
:102D60000139C9B2FF2900D110BD12F8013F002B73
:102D7000F6D05C1E01302340C0B2F8E7054B0022BC
:102D8000C3F808254FF44032C3F84423C3F80423A2
:102D9000704700BF00B00040044A1378591C1170FE
:102DA000012013B9024A1060184670473C06002003
:102DB00000B00040094B187828B9404080F31188D2
:102DC0004FF0040002DF0138C0B21870012310B9BF
:102DD000034A536070471846704700BF3C06002006
:102DE00000B00040014BD3F80405704700B000402C
:102DF00000F5A870014B43F82010704700B0004068
:102E0000114BF0B50124264600251A465E60C3F832
:102E10000405C3F80051C3F804511E60D3F8001133
:102E200031B9D3F8041119B9D3F804150029F5D133
:102E30005460D2F804110029E8D1D2F80475002FAB
:102E4000E4D0C2F80415F0BD00E0004070B58CB0CD
:102E50000E4615460146102268461C46FFF74EFFF7
:102E600010220DEB02003146FFF748FF6846FFF7DE
:102E7000C7FF25B1102208A92846FFF73FFF24B15C
:102E8000102208A92046FEF7EEFA0CB070BD000033
:102E9000024B1B6803B11847704700BF540800205D
:102EA000064B1860064B1022C3F80423054B022280
:102EB000C3F88021012006F0CBBB00BF54080020DE
:102EC0000010004000E100E008B5012006F0CEFB54
:102ED000034B0022C3F8FC2F0122C3F8FC2F08BDCE
:102EE000001000400228034B0CBF04220322C3F849
:102EF0001025704700100040014BC3F80C057047C7
:102F000000100040014BC3F8080570470010004056
:102F1000014BC3F854057047001000400A4A0023D3
:102F2000C2F82C350123C2F83035C378C2F82435F5
:102F3000437881781B0443EA0163017843EA012363
:102F4000C2F81C35704700BF00100040C2F34203B6
:102F5000022B10B50CBF4FF080740024D307C0F1D2
:102F600008034FEA034300F00F0003F4702340F41A
:102F70008070074A48BF44F48014034341F0007155
:102F8000234341F44031C2F81435C2F8181510BD7E
:102F900000100040014BC3F80405704700100040CA
:102FA000014BC3F80405704700100040014B01229B
:102FB0005A60704700100040014B01221A607047B0
:102FC00000100040034B0022C3F8002201221A61C6
:102FD000704700BF00100040064B0022C3F80021DC
:102FE000C3F80421C3F80821C3F80C21C3F8102149
:102FF000704700BF00100040014BD3F8000170473C
:1030000000100040014BD3F80C0170470010004045
:10301000034BD3F85005B0FA80F04009704700BF69
:1030200000100040044B40F20312C3F83425C3F8EB
:103030003805C3F83C15704700100040014BD3F829
:103040000004704700100040004870474C07002003
:103050000048704750070020024B0B22C3F80022A3
:10306000704700BF00100040024B0722C3F8002247
:10307000704700BF00100040024B0322C3F800223B
:10308000704700BF00100040034AD2F8003243F4FA
:103090008873C2F80032704700100040014BD3F82B
:1030A0004805704700100040024B0022C3F81C2165
:1030B000704700BF00100040014BD3F81C0170475F
:1030C0000010004030B50024A30003F1804303F555
:1030D00080531568C3F8005601349588C3F820560C
:1030E000082C02F10602EFD1024B40EA0120C3F89E
:1030F000400630BD00100040034AD2F8403623F0AD
:10310000FF03C2F84036704700100040034B002216
:10311000C3F81421C3F81821704700BF0010004005
:10312000014BD3F81401704700100040044BC3F862
:103130006005D3F8002242F04002C3F80022704735
:1031400000100040054B4FF48022C3F8482303F5DC
:10315000A033FF22C3F80825704700BF00B000402D
:10316000014BC3F84405704700100040F0B5A2F5CC
:103170007423234CA3F51073A34288BF02F1E872B5
:10318000204C214B88BF02F5D4324FF0000688BF97
:1031900002F5A5724FF00105B2FBF3F24FF0040304
:1031A000E560C4F80465C4F81035184B88BF01F118
:1031B000FF310227C4F80875C4F84025C4F84061FF
:1031C000C3F848154FF48021C3F84413C3F848618D
:1031D0000F4903F5A033C3F81815A1F5405108397C
:1031E000C3F81C45C3F80475C3F8101530B109497C
:1031F000C3F814151046C3F80455F0BD0649F7E7A7
:10320000BFBDF07F0080004040420F0000B0004092
:1032100048B100400010004004100040024B012261
:103220005A601A61704700BF008000400E4B0022B8
:10323000C3F84805C3F8482103F5B8330B4AC3F86F
:10324000302502F5DE424432C3F8342502F580729F
:10325000C3F83825A2F5E242383AC3F83C253022BB
:10326000C3F80425704700BF0080004004110040EF
:103270000B4B0C4AC3F8202502F5DE424032C3F85E
:103280002425A2F5DE423C3AC3F8282502F5DE42A9
:103290004032C3F82C250C22C3F80425704700BF28
:1032A00000F0014000110040034BD3F84405D3F86F
:1032B0004035C01A704700BF00800040064B074AE7
:1032C000C3F8482502F5DE423C32C3F84C25802283
:1032D000C3F80425704700BF00F001400C11004006
:1032E000014BD3F84805704700800040154B10B5DE
:1032F00000220224C3F80025C3F80045124CC3F88D
:103300000445C3F808051148C3F80C05C3F81015A7
:103310000F49C3F81415C3F800220E49C3F8002161
:10332000C3F80421C3F808210B4AC2F8401501F57F
:103330005F41C2F844154021C2F8041501221A6009
:1033400010BD00BF00F00040010000015007002048
:10335000400600200411004000F0014010B5104B61
:1033600000220224C3F80025C3F800454FF0807402
:10337000C3F80445C3F80805C3F80C1509480A4901
:10338000C3F81005C3F814150121C3F80012C3F8DF
:103390000021C3F80421C3F80821196010BD00BF43
:1033A00000F0004050070020400600200C4B022295
:1033B000C3F80423D3F804216AB10222C3F8082316
:1033C000084A4FF40041C2F88011D3F80801B0FA5E
:1033D00080F04009704720BF40BF20BFEAE700BF30
:1033E00000F0004000E100E0014BD3F8000470471A
:1033F00000F0004010B50E4C0123C4F800350D4B11
:10340000C4F80405C4F80815D3F80435C4F8103519
:103410000023C4F814354020FFF788FE064B074A06
:10342000C3F840254022C3F84445C3F8042510BD25
:1034300000F000400010004000F001402811004062
:10344000014BD3F80004704700F00040074BD3F85D
:1034500028213AB1064A0021C2F80011C2F804112D
:10346000C2F808110022C3F828217047001000405C
:1034700000F00040074BD3F8280148B103F5604342
:10348000D3F8000120B1D3F80401003018BF0120A7
:10349000704700BF00100040042905D8404080F369
:1034A00011884FF0040002DF084B03391860084B05
:1034B00001700122002181704170C3F80425C3F816
:1034C0000011C3F804231A60704700BF5808002099
:1034D00000D00040164B1A6830B50C188C42A4EB93
:1034E0000100537806D100200521013911F0FF01B8
:1034F00010D130BD95789D42F6D01344DB7804F8A6
:10350000013D537810780133DBB2984208BF0023A5
:103510005370E3E794789C4203D1064B01221A6072
:1035200030BD01331478DBB29C4208BF0023DCE7D6
:103530005808002000D00040154AD2F8003170B57C
:1035400023B3144B196888780D784C78431CDBB290
:10355000AB4208BF0023A34205D1012353600023DF
:10356000C2F8003170BD0844D2F80865C6708B708F
:103570000133DBB29D4208BF0023A3424FF000019C
:1035800008BF0123C2F8001108BF536070BD00BF1F
:1035900000D0004058080020F0B5037E05681A46A8
:1035A0000024FF2A01D10020F0BD02EBC2078A42AD
:1035B00005EB870615F8277004D0B3681C44134642
:1035C0003A46EEE7934200D107761BB203EBC30302
:1035D0003278B06805F823203378FF2B06D003EB50
:1035E000C30305EB83039A6802449A602044F0BD4C
:1035F00030B5551A15F4000F8468838A09D125F077
:103600007F4222449A420FD9D21A002382608382D9
:1036100030BD8A1A22F07F42944201D9A21AF1E702
:1036200013441B1B9BB200229B1A9BB20022EDE7A6
:1036300001460120FFF7DCBB01460020FFF7D8BBA5
:10364000032813D8DFE800F002090E1D01290DD16F
:103650000E4B02210020FFF713BA022906D10C4BB2
:103660000846F8E7012907D0022908D0404080F336
:1036700011884FF0040002DF064B0221F0E7064BF1
:10368000EEE70229F2D1054B0320E4E7B001002068
:10369000C0010020D0010020E0010020F001002046
:1036A00010B40C46032814D8DFE800F0020A0F21FA
:1036B00001290ED1114B0021002010BCFFF7E0B909
:1036C000022906D10E4B0121F6E7012907D0022974
:1036D00009D0404080F311884FF0040002DF094B0D
:1036E00000212046E9E70121074B0846E5E70229CA
:1036F000EFD1064B01210320DFE700BF600100206E
:10370000700100208001002090010020A001002015
:10371000404080F311884FF0040002DF08B5831E9B
:10372000012B01D9FFF7F4FF08BD012808B504D02B
:1037300005D3032804D0FFF7EBFF022008BD0120CA
:1037400008BD2DE9F047057F012304464377002D8E
:103750004AD1037EFF2B02D14577BDE8F087FFF702
:1037600041FB6769267ED4F80080C71B27F07F479E
:10377000FF2E06D006EBC60608EB86018B68BB421F
:1037800016D9A27AE37A934205D10133DBB2022B38
:1037900008BF0023E372E37A04EB83030122DD60B8
:1037A000002363770221636A1046BDE8F04718479B
:1037B000FF1A1D448A784B7818F826609B1ADBB2F2
:1037C000012BD5D1D1F80C90013A8A70B9F1000FD4
:1037D000CED060698B8A4A8B2844C01A20F07F4083
:1037E0000B69096AC847C3E7BDE8F0872DE9F04FC8
:1037F000427F8FB08046002A40F0A383436905933F
:103800000121837A0177C07A984200F088800B44C6
:10381000DBB2022B08BF002388F80A3008EB8303D1
:103820000091D3F80CB0059B5B4423F07F43C8F8AC
:10383000143098F818300393D8F800300293D8F871
:1038400004300A9398F809300193002306934FF04F
:10385000FF0A019B002B65D198F81830039A9B1A38
:1038600018BF01230493009BE3B1D8F80030DDF8C2
:103870000490029398F81860FF2E0CD037B2029B88
:1038800007EBC70703EB8704A5685D4540F2388165
:10389000A5EB0B05A560049B009A0399B14218BFE4
:1038A00013460493D8F800300193D8F804300C93F1
:1038B00098F809300293029B002B40F0748198F82D
:1038C0001830039A9342069B40F0328353B998F81C
:1038D0000940D8F80470013CE4B24FF02C0BFF2CE7
:1038E00040F09182002388F81C30049B4BB198F87B
:1038F0001830FF2B40F0DB82FFF75CFA08B9A8F81C
:103900001A0098F81D30002B00F01B830122D8F814
:103910002430114602200FB0BDE8F04F1847009246
:10392000934686E7019B03F1FF395FFA89F3019320
:10393000019A0A9B03EBC2077B680493F9782C2059
:10394000BE788E4285D0049B3C7816FB00F29D1811
:10395000731CDBB29C4208BF0023BB70049B9A5CC3
:10396000032AEDD9052A17D8697801EBC103099319
:103970000998029B03EB80046378A0781B1A13F06C
:10398000FF0309D0042A11D16A687AB9AA686AB912
:10399000EA6832F07F4209D100232B7001206B6A64
:1039A0002862002BCAD0A96A9847C7E7012B40F0CC
:1039B0009D804046FFF7F0FD2B78A060042B064663
:1039C00040F08680D8F814300793FFF70BFA079B76
:1039D0000890C31A23F07F435B449E4202469CBF7B
:1039E000A28A961B62689BBF9B19A382F31A0023CD
:1039F0008AB1A98979B101F1FF3E1FFA8EFEA5F8BF
:103A00000CE09A422DD3DFF80C93B4F81AC0E645C7
:103A100049D8A4F818E0AA8807991344A360EA8853
:103A2000A38A1344A382089A2046FFF7E1FD2A895E
:103A3000E38A13449BB2E3826A8993428CBF9B1A48
:103A40000023E382AB7B03B1E370029B099A03F886
:103A500022A0637895F801A00133637000202870DC
:103A60009DE7B4F81AC0E645CDD2216AA74EA84812
:103A70008E19864281BF01F1E87101F5D43101F55B
:103A8000A5712162266AE1698CBF4FF001094FF0F0
:103A90000009761A91440CF1FF3C2662A3EB09035E
:103AA000A4F81AC0ADE7266AE16999480E4497491F
:103AB000711881428EBF002101214E4411440CF146
:103AC000010C8CBF266226620B44A4F81AC09CE746
:103AD000A37863706B7898F819209A4201BFFF238E
:103AE00088F819300023A8F81A30B7E70221D8F86F
:103AF00024300122084698470123BE700693A8E6A9
:103B0000B8F81A309D4229BFFF235B1B88F8193093
:103B10000023A8F81A30E38AA9441BB188F8196079
:103B2000A8F81A300022029BA26013F8273088F808
:103B30001830D4F804E0BEF1000F30D0208BDFF84D
:103B4000D0C1236AE1690B447049591861459FBF90
:103B5000A3F1E873A3F5D433A3F5A573236292BF51
:103B6000009B23620023734410F1FF301A44E8D213
:103B7000059BA260D8F8141003EB09022046FFF75A
:103B800037FD238B63830023E370029B03F827A098
:103B9000637801336370ABEB050BB2466AE6A3783A
:103BA00063705646F7E7029B013BDBB20293029A31
:103BB0000C9B03EBC20305935B780093BAF1FF0FF4
:103BC00000F083800FFA8AF303EBC303019AD14616
:103BD00012F823A002EB83040025FF2323700FFAC1
:103BE00089F303EBC3039B000D930D9BD8F80020D2
:103BF000B8F81A0002EB030B98F81830DBF808103D
:103C000007934FF0FF0EFF2B07D003EBC30C02EB23
:103C10008C07BE68B14200F29F80BBF81660089620
:103C200006EB010C1E46FF2E40F0A480089F2FB12A
:103C30008142C0F0B880FF2E40F07F810798CBF81A
:103C4000081083428BF8003017BFBDF91CB088F80C
:103C500018900BEBCB0B02F82B90FF2B06D003EB4D
:103C6000C30302EB83039A68511A9960A378013366
:103C700063700020BAE00099BDF800200131C9B29C
:103C80002C2312FB03F30091059A059952680978D9
:103C90000098814208BF0020D15C0090032902EB0C
:103CA000030512D195F80190019909EBC90401EBC4
:103CB00084046078A17888420DD00021D1546B6AC9
:103CC000012028620BB1A96A9847059B009A9B784E
:103CD0009342D0D1EFE5EB6863602B69E361AB8A77
:103CE0002383EB8AE382AB69E360EB692361AB6812
:103CF000A3600026A6826A68D8F814102046FFF751
:103D000077FC012326626683E37066E75A2B17FF70
:103D1000592B177FB6562EFE6168002965D0236A9D
:103D2000E26989481344894A9A1882429DBFA3F1E7
:103D3000E873A3F5D433A3F5A573236298BF236278
:103D4000A3681944638B8CBF002201221144013304
:103D5000A1606383564646E0FF8A891B2FB138462F
:103D60009E46079312F82C304DE7864234BF801BE5
:103D70003846F6E737B207EBC7070B9702EB870722
:103D80000997BF680A9767450BD2099FFF8A002FE2
:103D90007FF44CAF0A9EACEB060C0B9E12F826602B
:103DA00041E7FF2642E7F1453FF460AFBEF1FF0F68
:103DB000B2D0764637B2019B07EBC70713EB870BF0
:103DC000AAD0E2789BF803309A42A5D93146404602
:103DD000FFF7E2FB9BF802308BF80130019BCBF838
:103DE000080003F827A0B246FFE60120002D3FF4AB
:103DF000E5AE00232B706B6A2862002B3FF4DEAE29
:103E0000A96A9847DAE607EBC4056B78EA789A4224
:103E100002D1013CE4B262E513FB0BF269688B1836
:103E20008A5C012A2FD0022A08D06B782A780133C5
:103E3000DBB29A4208BF00236B70E6E7D3F804C0F8
:103E40009A689CF80010D3F80C90D8F80000D8F8C5
:103E500014A0FF2902D0166856451DD098F81810F6
:103E6000C2F800A00022FF2909D001EBC10A00EB33
:103E70008A0EBEF81660DEF808E0A6B172448CF82F
:103E80000010C9F8002000221A625A6A002ACCD019
:103E9000996A186A9047C8E701EBC101D9F8002078
:103EA00010F82110DFE7724410F82A10DBE7039BBB
:103EB000FF2B07D1FEF796FF0446FEF76DFF08B90A
:103EC000C8F8144098F81830D8F8002003EBC30362
:103ED00002EB83030A269D68FEF784FFD8F814409E
:103EE000031B23F07F430333AB422CBFE418641958
:103EF00024F07F440746D8F8283020469847FEF73C
:103F000071FFC01B20F07F40E41B033024F07F448E
:103F1000A0427FF6F6AC013EDED1404080F311882E
:103F20004FF0040002DF9DF8083088F81C30DEE412
:103F3000002BF8D101230493C9E4B1457FF43AAFD3
:103F400094E60FB0BDE8F08F592B177F5A2B17FF5F
:103F5000F0B5059F9DF8184018B1012828D0012020
:103F6000F0BD1D4D1D4E2E621D4E6E621D4EAE6289
:103F7000194D2C2606FB00FC05EB0C0E45F80C2019
:103F80008EF8081007998EF80930CEF80470013BBE
:103F9000DBB2FF2B14D1002CE1D12C2202FB00500C
:103FA00003764376448344618472C4722046F0BD34
:103FB000094D0D4EEE640D4E2E650D4E6E65D7E724
:103FC0001AB207EBC20ECEF8041017F83220A41A6A
:103FD00002FB0611E4B2DAE75C0800202B37000090
:103FE000A1360000393600001D37000041360000C0
:103FF00031360000054A2C2303FB0020436A1BB125
:104000000122114600201847704700BF5C080020BD
:10401000F8B5224D2C2404FB00500FFA81FCD0F897
:1040200004E00EEBCC071EF83CE0FE78751CEDB208
:10403000AE4598BF002597F801E0AE452BD0D7F8E4
:1040400004E016FB04F60EEB06044FF0030C0EF82A
:1040500006C06360069BA360079BE360089B236127
:10406000BDF82830E382BDF82430A3820B9BA36106
:104070000C9BE3610D9B636202260E9B6270A36240
:104080002662FD70456A036A084698470022314659
:10409000A847206AF8BD0120F8BD00BF5C080020D9
:1040A000F8B5214D2C2404FB00500FFA81FCD0F808
:1040B00004E00EEBCC071EF83CE0FE78751CEDB278
:1040C000AE4598BF002597F801E0AE452AD0D7F855
:1040D00004E016FB04F60EEB06044FF0040C0EF899
:1040E00006C0A380BDF81830E380BDF81C302381E2
:1040F000BDF820306381BDF82430A3819DF82830BD
:10410000A3730B9B636202260C9B6270A362266200
:10411000FD70456A036A0846984700223146A84761
:10412000206AF8BD0120F8BD5C080020F8B5194CE4
:104130002C2505FB00400FFA81FCD0F804E00EEBC3
:10414000CC071EF83CE0FE78741CE4B2A64598BF8C
:10415000002497F801E0A64519D0D7F804E016FB33
:1041600005F60EEB06054FF0050C0EF806C06B6267
:104170000226069B6A70AB622E62FC70446A036A78
:104180000846984700223146A047286AF8BD01201A
:10419000F8BD00BF5C0800202DE9F0411C4D2C2427
:1041A00004FB00500FFA81FCD0F804E00EEBCC07C2
:1041B0001EF83CE0FE78751CEDB2AE4598BF0025B8
:1041C00097F801E0AE4520D0D7F804E016FB04F6DE
:1041D0000EEB06044FF002080EF80680A360069B63
:1041E000E360079B6362FF26089B62606670A362C0
:1041F000C4F82080FD70456A036A0846984700228B
:104200004146A847206ABDE8F0810120BDE8F08161
:104210005C080020F8B5194C2C2505FB00400FFA6E
:1042200081FCD0F804E00EEBCC071EF83CE0FE78F1
:10423000741CE4B2A64598BF002497F801E0A64597
:1042400019D0D7F804E016FB05F60EEB06054FF083
:10425000010C0EF806C0FF266E7002266A62AB6281
:104260002E62FC70446A036A084698470022314671
:10427000A047286AF8BD0120F8BD00BF5C080020F7
:10428000074A10B52C2303FB0020446A036A084642
:104290009847234600220221BDE81040184700BF7E
:1042A0005C080020FEF79EBD401A20F07F4070475A
:1042B00070B50C4D06460C460CB9002070BD4FF091
:1042C000FF31284605F00EFD20463146FFF702F982
:1042D0000446284605F06AFD002CEED020BF40BF02
:1042E00020BFE9E73004002020BF40BF20BF704757
:1042F0000860704718B90B6843F000430B607047C3
:1043000018B90B6823F000430B60704770B502FBCF
:10431000011102789DF810500A44252192FBF1F416
:1043200001FB1424E1B2CA0801709A5C04F007048E
:10433000224112F0010209D1B1FBF5F005FB10108A
:10434000C0B25D1E04339D4202D11146084670BDC5
:1043500015F8016F00241119082CC9B201D10A46C1
:10436000F1E716F0010F03D00028EFD00138C0B2FA
:1043700076080134EFE7000010B50E4A92F8463295
:1043800092F845128B4238BF92F8444292F8451297
:1043900038BF1B195B1ADBB298429FBFD2F840327C
:1043A00092F8451253F82100012394BF03710020B5
:1043B00010BD00BF0409002070B590F8581090F8A7
:1043C00059308B423FD190F8343013F0010511D0B1
:1043D00090F88C309B0738D590F88D30082B34D965
:1043E000B0F88E304FF6FF7293422ED1B0F8902085
:1043F0009A422AD1C48C828CA0F85E40848DA0F8A9
:104400005C20002354437D2201269D4202FB04F2DE
:104410004FF47A7492FBF4F2A0F8602090F88520B3
:1044200080F884600CBF3446022464F3020266F311
:10443000C4020139C36780F8852080F8591080F8DC
:104440005A60184670BD012070BD022070BD00008A
:104450002DE9F84F0C78944281460F4690463DD0A6
:104460001F4ED6F8743233F83430038000254FF0F5
:10447000020B06F51A7A22B2D6F87402B9F800E0F7
:1044800000EBC20130F83220964520D1486801285F
:1044900020F003030AD9F3B1021D1CD04279D2B136
:1044A000027902F00302013A012A14D801221544CC
:1044B0004A60EDB213B15146FEF703FC013496F8A1
:1044C0007822E4B2A24208BF00244445D3D13C7014
:1044D0002846BDE8F88FC1F804B0EBE70025F7E700
:1044E0000409002010B5094B93F81C2282420446AF
:1044F00009D90246FC21D3F81402FEF7F7FB10B1EC
:10450000038CA34200D0002010BD00BF040900208E
:104510002DE9F04186B0022305280546884602931E
:104520000CD006281AD013D9073880B2FFF7DAFF6B
:10453000002800F0BB8090E8C00004E05C4BD3F89A
:10454000C460D3F8C8705A4CA37B03F0FF005BB182
:10455000404080F311884FF0040002DF544BD3F841
:10456000AC61D3F8B071EEE702AB00932A46514B31
:10457000A5730321FFF7DAFD022849D0029B002B27
:1045800040D1237B9D4202D0637B9D4236D106AB56
:10459000022243F80C2D002200930321454B1046C4
:1045A000FFF7C4FD022807D1012211460320FEF7C0
:1045B0003FFA039B022BCBD003980222002843D161
:1045C00006AB032143F8082D01220093394BFFF776
:1045D000ADFD022807D1012211460320FEF728FA7B
:1045E000049B022BB4D0049A02BBB7422AD9324BA7
:1045F00011460320FEF744FA0028A9D1A37B0BB98A
:10460000012302930023A373029806B0BDE8F08152
:10461000637B9D4204D1012211460320FEF708FA74
:10462000029B022BAAD1FFF75FFEF9E7049B012B47
:104630008ED100221146204B0320FEF721FA0246BC
:10464000002885D11D4BD3E7039D012D80D106ABFA
:10465000032143F8042D002000934246154BFFF739
:1046600065FD022808D12A4629460320FEF7E0F915
:10467000059B022B3FF46CAF059B1BB1059B012BE7
:104680007FF466AFE37B002BB8D00D4B04229A6019
:10469000002211460320FEF7F3F900287FF458AFFB
:1046A000E37B002BAAD0FFF71FFEF9E70120ACE760
:1046B00004090020F142000020020020A002002096
:1046C00040020020F8B590F8A430D0F8E850044635
:1046D00018060E4605F104021ED4EDB119074CD59B
:1046E000002A4AD06979002947D0297901F00301CD
:1046F000032911D194F8341011F0010F03F0400197
:10470000EB792CD131BB022B37D0112B04D82F4998
:1047100021FA03F3DB0730D494F8A43043F080038C
:1047200084F8A430FEF790FC0378012262F30103C1
:1047300000224270D4F8E8200370DBB2D2B143F01B
:104740001003037003786FF3471303700023837023
:104750003060F8BD991E01290FD90B2BD4E729B978
:10476000022B0AD0112BD7D81949D1E7022B04D03C
:10477000042BF6E762F30413E3E794F8F93094F8B6
:10478000F810D01811B9417884F8F81023B1D15C31
:10479000012767F30101D15494F8F810C91AC9B27E
:1047A0004170D45C1B296FF30414D45405D91B2128
:1047B0004170D15C41F01001D15429680029C1D069
:1047C000D15C41F01001D154BCE700BF4020020091
:1047D00060200200000000002DE9F04F8FB08146FC
:1047E000069303680991002B90462EDA816842688F
:1047F00023F0004391422CBF5B1A9B1A00240793BD
:10480000FF238DF82930ADF82A400B940C940593C2
:104810009A46A3462546089402230D930DAB0293B6
:10482000714B01930CAB00930DF129020BAB0121ED
:104830000020FFF7B1FC02280DD00D9B7BB140405A
:1048400080F311884FF0040002DF0023D6E7012136
:104850000020FFF715FD0D9B022BF8D0EDE79DF82A
:104860002920FF2A56D0BAF1FF0F03D00B9B0899DD
:104870009942E4D1042A49D9062A40F28B80059B4B
:10488000FF2B47D1594B073A92B2FC21D3F81402BF
:10489000FEF72CFA8145074638D0099B1BB990F8E2
:1048A0003430DB0732D4079B0C9E1E443B68002B40
:1048B00008DABA68796823F000438A422CBFB61838
:1048C0007618F61AD8F800309E4217D99D4238BFA4
:1048D0001D460BF1640A189B1B78A34207D9294691
:1048E0003046FFF7E1FCFB68534498422DD2BDF8F7
:1048F0002A30069AC8F8005093420BD20B9B0893BB
:10490000FB689DF829A003F1640B3546189B1B78C2
:10491000A34281D89DF82930FF2B11D1D8F800305F
:10492000DFF8CC902EA7D7E900679D4238BF1D461F
:104930004FF0070A189B1B78A3422DD8C8F80050E7
:10494000189B1C700FB0BDE8F08F294A05EB0B03D4
:10495000A3FB0201072202FB031121A3D3E90023D9
:10496000FBF758FC40F2E243B0FBF3F0069B80B249
:104970009842ADF82A000BD2199B022203EB4400A7
:104980000DF12A010134FCF76EFDE4B22835A2E7EF
:104990000025ACE70592B9E705EB0B03A3FB090182
:1049A0000AFB031132463B46FBF734FC40F2E2437C
:1049B000B0FBF3F0069B80B28342ADF82A000BD91E
:1049C000199B022203EB44000DF12A010134FCF78C
:1049D0004AFDE4B22835ADE70025AFE7AFF300802C
:1049E00000CA9A3B00000000F142000004090020C8
:1049F0008D49FD1A000000002DE9F041044688B001
:104A0000B0F8662034480623A2FB00018DF80D3073
:104A100040F2231303FB02112DA3D3E90023FBF77C
:104A2000F9FB08AA0DF10D0105AE42F8100DB4F81E
:104A30005C300091019601212046FFF7CDFE04F184
:104A4000660504F172074FF6FF78022229460DF140
:104A50000E00FCF708FD9DF80D00BDF80E200023A8
:104A6000D9B288421ED80235AF42EED194F8583000
:104A700084F85930194B0022C3F88C22D4F88030C6
:104A800013F8052C42F0030203F8052C032203F867
:104A9000042C112203F8022C0F2203F8012C2022EF
:104AA0001A7012E0424503D036F81310914201D03B
:104AB0000133D5E740F2E2435343E36702220DF1AD
:104AC0000E01D4F88000FCF7CEFC08B0BDE8F08100
:104AD0008D49FD1A070000000054CE09040900208A
:104AE0001FB50023039306238DF80B3090F8343064
:104AF000DB0742BF0246436D42F8783FD0F8801092
:104B000001910DF10B01009158BF03AAB0F85C3080
:104B10000021FFF761FE05B05DF804FB0000000016
:104B20002DE9F04F8BB00024FF25DFF804B18DF89C
:104B30001F508046894692461F461C6008942646B0
:104B40000AAB022243F8042D0293374B019308ABC2
:104B500000930DF11F02534641460020FFF71CFB56
:104B600002280BD0099B6BB1404080F311884FF0B5
:104B7000040002DF41460020FFF782FB099B022B65
:104B8000F8D0EFE79DF81F20FF2A45D0062AD7D995
:104B9000073A92B2FC21DBF81402FEF7A7F80346AD
:104BA0000028CDD090F83420D207C9D4D0F800E046
:104BB000089ABEF1000F09DA416880682EF0004EB5
:104BC00088422CBF12185218A2EB0E02FF2D05D1FD
:104BD000DC689DF81F5027341646B1E73146104671
:104BE00005930492FFF760FB09F10201214488421A
:104BF000049A059BECD90D483444A4FB000107231B
:104C000003FB041106A3D3E90023FBF703FB2030C9
:104C100038600BB0BDE8F08FFF2DECD1F9E700BF95
:104C200000CA9A3B00000000F14200008D49FD1AC5
:104C3000040900200000000073B5164602AA0546CC
:104C400042F8046D012027311C46FFF769FF0198E7
:104C5000864211D03146FFF727FB02461048072352
:104C6000A2FB000103FB02110BA3D3E90023FBF716
:104C7000D1FA2368184420602368002B05DB40F23A
:104C8000E24068432368984201D302B070BD1B1A0A
:104C90002360F7E7AFF3008000CA9A3B00000000F2
:104CA0008D49FD1A13B500F17C030446426FC168BB
:104CB000808CFFF7C1FF02A9E36FD4F8800040F2B7
:104CC000E242B3FBF2F3022221F8023DFCF7CBFBF8
:104CD00002B010BD0B4A92F8843292F885129942C4
:104CE0000ED192F8843202EB4303A3F87E0292F8CD
:104CF00084320133DBB2032B08BF002382F88432F5
:104D0000704700BF04090020044B1B7C23B1012124
:104D100000220846FDF78CBE704700BF0409002042
:104D200008B50A4B00221A7068B1012805D1084B5A
:104D300000221146FDF7A4FE38B1404080F31188EF
:104D40004FF0040002DF034BF2E708BDE80D00203E
:104D5000900200208002002038B505460C46002154
:104D60000846FEF7BFF895F8A430DB064FF00102C5
:104D70000CD51F210820FEF7E9F8214605F1A50012
:104D8000FEF7B4FABDE83840FEF704B908201B214D
:104D9000FEF7DCF82046F5E738B505460C4600215D
:104DA0000846FEF79FF895F8A4309B064FF00102E5
:104DB0000CD51F210820FEF7C9F8214605F1C600D1
:104DC000FEF7CCFABDE83840FEF7EAB808201B2110
:104DD000FEF7BCF82046F5E7404080F311884FF01D
:104DE000040002DF30B50468002C89B019DA43688A
:104DF000856806909D4224F0004434BFE41A641B89
:104E0000094B0593A4B2002304930393029318461D
:104E100001940094FFF744F930F0020301D0FFF74A
:104E2000DBFF09B030BD00BF0143000003460A4666
:104E3000D3F8981010B5983009B9FFF7CDFF1C8C46
:104E4000A3F89E4083F8A02004240B4A83F89C40DA
:104E500092F87C4283F8984002F51572FDF760FFE6
:104E600028B9404080F311884FF0040002DFBDE80C
:104E7000104003F0A3BB00BF0409002010B5164A80
:104E800092F8453292F84612994201D1FFF7A4FFF9
:104E900092F84512D2F8403253F8210092F87C3251
:104EA0000168037092F8453292F844420133DBB254
:104EB0009C4208BF002382F8453202F51572FDF7C7
:104EC0002FFF28B9404080F311884FF0040002DF23
:104ED000BDE8104003F072BB0409002037B541F271
:104EE000D6230021009308461C4B0522FFF71EF92C
:104EF00030F0020105D0404080F311884FF00400EB
:104F000002DF4FF4975300930122144B0846FFF73A
:104F10000DF930F00202EED141F2E5230093114683
:104F20000E4B1046FFF702F930F00205E3D10120E5
:104F3000FFF722FA04460028DDD04FF6FF73C38046
:104F400003230371182229460B30FCF7B8FA3C23DF
:104F5000E37203B0BDE83040FFF790BF1D5500007D
:104F600070B506460320FFF707FAA0B14FF6FF73AE
:104F7000447AC3800223037100F108051C4446B142
:104F8000FEF78CF800F07F002855FFF777FF002030
:104F900070BD7F20F8E7012070BD262810B50446BB
:104FA0000BD027280BD025280BD10220FDF7AAFF14
:104FB0002046BDE81040FDF7ABBF1A20F6E75020B1
:104FC000F4E70A2802D802304000EFE7272801D88A
:104FD0000330F9E7FFF700FF38B51C4C94F8553162
:104FE00094F856219A4206D00133DBB2022B08BF57
:104FF000002384F8553194F85501272303FB004022
:1050000000F20710FDF7CCFF9620FEF7A9F8FEF797
:1050100023F894F8D430C3F3C202D3B21946002067
:1050200011F0010F00F101050DD0013B134094F880
:10503000D420C0B263F3C50284F8D4202530BDE883
:105040003840FFF7AABF49082846E9E704090020CD
:1050500038B5104A92F87C3292F878420133DBB2CC
:105060009C4208BF002392F87B429C4201D1FFF78B
:10507000B3FE92F87C52D2F8744224F8350092F8CC
:105080007C0204EBC004616082F87C32BDE83840E9
:1050900003F094BA040900202DE9F843244C064695
:1050A00000272EB194F8793294F87A229A4201D1ED
:1050B000BDE8F88394F87982D4F87092D4F8140299
:1050C00039F8382009EBC803FC215D682F60FDF733
:1050D0000DFE034639F838001A8C82421FD1D3F8EE
:1050E000F02042B9D3F8E820C3F8F0501AB9C3F859
:1050F000E850C3F8F420D3F8F42002B11560C3F8E7
:10510000F45094F8793294F878220133DBB29A4261
:1051100008BF0023013E84F87932F6B2C1E72B794B
:1051200067F301032B712946FFF792FFE9E700BF00
:105130000409002073B50122044611460020FDF742
:1051400077FC94F82020002141F6E63307320093E3
:105150000846384BD2B2FEF7E9FF30F0020105D025
:10516000404080F311884FF0040002DF324B1A7C7C
:10517000052A1D461AD11A7B238C07339A4215D172
:1051800041F6F233009301222A4B0846FEF7CEFF88
:1051900030F00202E4D141F6F93300931146254B79
:1051A0001046FEF7C3FF30F00203D9D1D4F8E8105F
:1051B000D4F8EC30994203D0D4F8F030994201D1C0
:1051C0001E4E12E00B796FF301030B710B68C4F8EC
:1051D000E830208CFFF73CFFE8E70368C4F8E830CC
:1051E000C4F8EC303146FDF76CFDD4F8E80018B196
:1051F000D4F8F0309842F0D10023C4F8EC30D4F861
:10520000E81051B94FF6FF732384D5F88C329C42D5
:1052100008BFC5F88C1202B070BD0B796FF30103A3
:105220000B710B68C4F8E830C4F8F030208CFFF73D
:105230000FFFE4E71D55000004090020640B002067
:10524000C0B208B5031F012B01D9FFF7C5FD084AFD
:10525000137C3BB1043B012B04D91074BDE808401A
:10526000FDF7B0BEFDF7D4FE0028F7D008BD00BFA3
:105270000409002008B50A4A137838B1591C117086
:1052800063B90120BDE8084003F096B90BB9FFF7F8
:10529000A3FD013BDBB21370002BF3D008BD00BFB0
:1052A000840D00200020FFF7E5BF0000002208B5B4
:1052B0001146044B1046FDF7E3FB08B1FFF78CFDE8
:1052C00008BD00BF60020020002208B51146044B53
:1052D0001046FDF7D5FB08B1FFF77EFD08BD00BF06
:1052E00000020020064A08B59360134600221146CA
:1052F0001046FDF7C5FB08B1FFF76EFD08BD00BF06
:10530000300200202DE9F04F14681D688DB0002C8C
:1053100080460B9117469A469DF85C9003DA169CDE
:10532000AC4238BF2C46AC424F4E1BD941F2C703AA
:1053300008934E4B05930021631B00930796434649
:105340000691049103910291019101220846FEF712
:105350005FFE30F002032BD0404080F311884FF005
:10536000040002DF1DD200231A4619461846FFF733
:10537000ABFF41F2DC03002108932C1B3C4B05934F
:10538000079643460691049103910291019100947E
:1053900001220846FEF73CFE30F00203DCD12C4629
:1053A0000BE000231A4619461846FFF78DFF00232D
:1053B0001A4619461846FFF779FFDFF8BCB00B9B79
:1053C000CBF8083041F2F4030893199B06930022AE
:1053D000189B059304920392029201921146104683
:1053E000079600944346FEF713FE30F00202B3D155
:1053F000052311461046FFF775FFDBF888329D4202
:1054000021D03A68CAF8003022F000429A4238BFF0
:105410001A463B68002BB8BF23F0004341F221112C
:10542000B8BF3B6092B2A3B20691002102930192F1
:1054300000920596049103914A460846FEF730FE15
:1054400030F0020388D1FF20FFF726FE094B01222E
:1054500011460020C3F80890FDF712FB00287FF4E6
:105460007BAF0DB0BDE8F08F1D550000C9520000A4
:10547000AD520000B0020020040900201FB5094A07
:105480000523002413730394074C02940193D2F86C
:10549000CC30009302F1C803C432FFF733FF04B0ED
:1054A00010BD00BF040900204157000008B530B10D
:1054B000034B9B7BC9B2994201D0FFF78DFC08BD1D
:1054C0000409002008B528B1034B9B7B052B01D0B4
:1054D000FFF782FC08BD00BF04090020012808B5C1
:1054E00008D1054B9A7B062A02D100229A7308BD87
:1054F000FFF772FC08BD00BF04090020012808B5B1
:1055000008D1054B9A7B052A02D100229A7308BD67
:10551000FFF762FC08BD00BF0409002008B508B110
:10552000FFF75AFC08BD000013B502AC0E4B44F85F
:10553000043DFDF7C9FC0020FDF7DEFC0B48FDF73C
:10554000AFFC00210846FDF7CDFC2046FDF7E6FC48
:10555000002225210820FDF7F9FC054940F25B6097
:10556000FDF760FD02B010BDD6BE898ED966000081
:10557000555555002DE9F843214D95F8464295F8CB
:10558000443295F858920134E4B2A34208BF002493
:1055900005F5137705F50D78B9F1000F03D095F8EF
:1055A00045329C4201D1BDE8F8833846FDF76FFBD8
:1055B00006460028F7D04046FDF769FB28B930467B
:1055C0001049BDE8F843FDF77CBB066095F846221C
:1055D000D5F8403243F8220085F8464295F8443227
:1055E0000134E4B2A34208BF002495F8583209F10F
:1055F000FF39013B85F858325FFA89F9CCE700BFE3
:1056000004090020500B002010B52E4C94F81C22E9
:10561000002A36D004F50673FC21D4F81402FDF7F5
:105620000FFB294B94F83E22B4F83C12D4F8300218
:10563000FDF706FB94F8441294F81C22234BD4F88F
:1056400048020A440821FDF7FBFA214BD4F85C021A
:1056500002222421FDF7F4FA94F87822D4F86402A7
:105660001C4BB4F86C12013A92B2FDF7E9FA1748F4
:10567000FDF70DFB40B9404080F311884FF0040066
:1056800002DFC4F81822CCE7134A111FFDF745FBCF
:1056900094F8D43043F0070384F8D430FF2384F81F
:1056A000263284F8273284F8283284F829321F23DE
:1056B00084F82A32252384F82B32BDE81040FFF706
:1056C00059BF00BF04090020380B0020500B0020F8
:1056D000640B00206C0B0020580B0020024B186854
:1056E000436800211B68184704090020024B186812
:1056F000436800215B6818470409002070B5144610
:105700000E460546FEF7CEFD2146FEF7CDFDC41C34
:10571000092C11D9094B1B7813B10020FFF700FBAE
:10572000324600212846FFF75DFBAB681C44262C5F
:1057300000D8AC60012070BD002070BDE80D0020D5
:1057400038B5264BDA7B054602F0FF011C462AB12C
:10575000404080F311884FF0040002DF1B7BDBB276
:10576000052BF5D10122E2730222217322746373A7
:105770006060FFF7D9FE94F8D420134662F3C503A6
:1057800084F8D430FFF728FC94F8D43013F0C00F1D
:1057900007D004F1D70294F8D61094F8D500FDF79D
:1057A00091FCA26805F109010120FDF7DFFCFDF77E
:1057B00085FD2A4605210A48FFF7A0FF034628B1C8
:1057C00004232374BDE83840FDF7FCBB054A0146BD
:1057D000FEF720FD30F00203BAD138BD04090020E5
:1057E000C8090020094D000010B50446FDF76CFB08
:1057F0000020FDF781FB0A48FDF752FB04F1100081
:10580000FDF78CFB637DA17D1B0243EA0143217DF3
:1058100040F25B601943BDE81040FDF703BC00BFD8
:10582000D9660000F0B5384D1C46EB7B85B00646C6
:1058300003F0FF022BB1404080F311884FF00400C9
:1058400002DF2B7B218CDBB207318B42F3D185F851
:10585000242285F82522DBB20427EF732A736B73A9
:10586000238DC5F8204202206385228528746E604E
:10587000FFF712FC03A92046FEF724FF039994F8D2
:10588000A4200B7862F3C303C2F3400262F38203E5
:105890000B702046FFF7A8FF03992046FFF77CFA1C
:1058A0009620FDF75DFCFDF7D7FB237F5A06C2D497
:1058B00003F03F03628DA17F009304F11F0004F108
:1058C0001703FEF723FDFFF768FBAA6806F109013D
:1058D0000120FDF74BFCFDF7F1FC94F82010073197
:1058E0003246C9B22046FFF709FF034620B12F74A4
:1058F000FDF768FB05B0F0BD044A0146FEF78AFCDF
:1059000030F0020397D1F5E704090020094D0000AB
:10591000F7B5424D1C46EB7B064603F0FF022F46CF
:105920002BB1404080F311884FF0040002DF2B7B45
:10593000218CDBB207318B42F3D185F8242285F824
:1059400025220321DBB2E9732A736B73238DC5F81B
:105950002042012168606385228520462974FFF773
:1059600043FFD5F8403295F8452253F822102046DF
:105970000831FFF7F1F99620FDF7F2FBFDF774FB14
:10598000237F13F04005CCD103F03F03628DA17F4C
:10599000009304F11F0004F11703FEF7B7FCFFF7B3
:1059A000FCFA636C226C25641344E26B63649342DB
:1059B00088BF6264E36CA26C0020134406F1090105
:1059C000BA68E364A064FDF7D1FB0546FDF750FC1F
:1059D000E36C606CF23303EB40002844FDF726FCD7
:1059E000FDF76CFC94F8201007313246C9B220460E
:1059F000FFF784FE034648B104233B74FDF7E2FA47
:105A0000022003B0BDE8F040FFF746BB044A014660
:105A1000FEF700FC30F0020383D1F1E70409002017
:105A2000094D000010B590F8A440D0F8EC3014F007
:105A3000800F22D1D0F8E820FAB1240701D59A428C
:105A40001BD1D0F8F040A24204BF1468C0F8F04067
:105A50004BB913680B601160C0F8EC100B680BB900
:105A6000C0F8F41010BDD0F8F0201C68944202D1A8
:105A70000A601960F2E72346F7E72BB9D0F8E8305F
:105A80000B60C0F8E810E7E7D0F8F0201C689442FB
:105A9000EED02346FAE7000010B50B460446A9B93C
:105AA0000C48FDF7F4F8014608B9FFF795F9031D16
:105AB0001A7842F003021A7001225A700622DA7034
:105AC00031B12046BDE81040FFF7ACBF0021EFE741
:105AD00010BD00BF640B002010B504460948FDF757
:105AE000D6F8014608B9FFF777F9037943F00303C5
:105AF0000371012343710B23C3712046BDE810409D
:105B0000FFF790BF640B00202DE9F04F1C4693F87F
:105B100020309B4D0733DBB28DB02B7394F83430BB
:105B20000A91D907804609D5A36B216C02FB033388
:105B30000B44E16B23648B4288BF2164268D94F86B
:105B400058303244668C92B22285324496B294F830
:105B500059209A4200F0ED8200220523114610469A
:105B6000FFF7C0FB94F85A30013B042B00F2BC80D5
:105B7000DFE813F005008302200319044804D5F878
:105B80008C220AB9C5F88C4294F8853013F00703CB
:105B900000F0028112B1944240F0CB82043B012B11
:105BA00040F2C7827748FDF772F80746002800F0F8
:105BB000C08294F8853003F00703032B3DD194F89D
:105BC0003430DB0741D594F8583084F8593000233D
:105BD000C5F88C323B7943F003033B7118237B718A
:105BE0001023FB71B4F85C303B817B81B4F85E30EC
:105BF000BB81B4F86030FB8194F862303B74B4F838
:105C00006430A7F81130B4F86630A7F81330B4F850
:105C10006830A7F81530B4F86A30A7F81730B4F830
:105C20006C30A7F81930B4F86E30A7F81B30B4F810
:105C30007030A7F81D30394644E2022B5AD0032BAE
:105C4000C1D0012B50D1504900E0504994F8342084
:105C500012F001024ED194F8853062F3020384F809
:105C60008530E38C063333449BB2A4F86430387932
:105C7000FA7140F0030038710C20787194F8842098
:105C80003A72E26F40F2E240B2FBF0F2A7F809206C
:105C9000B4F85C20A7F80B20B4F85E20A7F80D201C
:105CA000B4F86020A7F80F20A7F811302268C4F8D4
:105CB0007480002A0ADAA368606822F000428342F6
:105CC0002CBF434408EB00039B1A636707F10903E9
:105CD000C4F880302E4BD9600122114600209C6010
:105CE000FCF7CEFE0028A6D0404080F311884FF08C
:105CF000040002DF94F88530052262F3020384F881
:105D000085303B7943F003033B7118237B710F23EC
:105D1000FB71B4F85C303B817B81B4F85E30BB81B1
:105D2000B4F86030FB8100233B74FB743B754FF08B
:105D3000FF33A7F811607B75BB75FB753B767B76EF
:105D4000BB76FB763B777B77BB772268238E6386B7
:105D5000002AC4F874800ADAA368616822F000425D
:105D60008B422CBF434408EB01039B1A636707F186
:105D70001303C4F88030064B064ADA60ACE700BF74
:105D800004090020640B0020A54C0000F949000024
:105D900050020020E14A0000B4F86470F71BBFB263
:105DA000380400F1C68194F8582084F85920D5F8B9
:105DB0008C222B73944208BFC5F88C32E26D636A63
:105DC0009A420CD1A38DA28CB4F860105A437D2363
:105DD00053434FF47A7293FBF2F3994216D00220A8
:105DE000FEF7CAFA00283FF47FAF238CC380052357
:105DF00003710023C372B4F85C308381B4F85E3061
:105E0000C381B4F860300382FFF738F82368D4F810
:105E100004A0002B09DAA06823F0004350452CBFF2
:105E20008044D0442360A8EB0308A38CB4F85C60E2
:105E3000A94913FB07F39BB2B3FBF6F21FFA82F9F1
:105E400016FB09F080B2834280F0FB80C01A40F25A
:105E500023124243C31701FB0323A0FB0101194492
:105E60009BA3D3E90023FAF7D5F920F07F4000EB9C
:105E700008030A93238DD4F87CB0DB1B4B442385A5
:105E800023689A4538BF9A4694F83430CDF82CA050
:105E900040F2E24813F0010F08FB06F6DFF85CA2BF
:105EA00000F0E080A26B216CC3F3420302FB1717E2
:105EB00095F82C12894A32F8115032F813301D44EB
:105EC000754305F57425864B05F23F25B5FBF3F5C3
:105ED00094F88430A56308FB03F305FB09F072080E
:105EE000963AA36407440023974294BF2764226430
:105EF000E2636365A0FB0A0175A3D3E90023FAF707
:105F000089F90A9B1B1ABBFBF8F008FB00F00A9307
:105F1000A0FB0A016EA3D3E90023FAF77BF994F8FA
:105F2000853003F01803102B20F07F48A6EB050501
:105F300002D12046FEF740FAB4F85C30B4F8602095
:105F4000A384B4F85E30E38442F210735343B3FB8E
:105F5000F6F3A385634BB3FBF6F694F885302686FB
:105F600013F0180308BFE3850121002002F0F0FAC6
:105F70000022012181461046FCF75AFD94F82020AA
:105F800041F26553002107320093D2B2564B0846C6
:105F9000FEF7CCF830F002077FF4A6AEA5FB0AAB03
:105FA0004BA3D3E9002350465946FAF733F94F4A39
:105FB00094F8206020F07F45072320F07F400021E7
:105FC000434302FB0133A0FB0201BAEB000019447A
:105FD0004FF47A724FF000036BEB0101FAF71AF9F4
:105FE0000B9AE3684249029013449AB294F8343011
:105FF000049213F0010F06F107063E4B069408BF0A
:106000000B4641F275510891F6B237490791059355
:1060100003970195CDF800800A9B324639463846F1
:10602000FDF7F6FF30F002007FF45EAEB9F1000F2D
:1060300000F0BD80012211460DB0BDE8F04FFCF725
:10604000F7BC06FB123292B2A2FB010140F223130D
:1060500003FB02111EA3D3E90023FAF7DBF8A8EB38
:10606000000306E71AA3D3E90023ABFB0A01FAF702
:10607000D1F8354620F07F485EE794F85C30002B7D
:106080003ED01D48FCF703FE0546002851D00023F2
:1060900084F85C30E38C06333344A4F8623003792F
:1060A00043F003030371082343710123C37104F117
:1060B0005D0105220830FBF7D6F9B4F86230A5F887
:1060C0000D3029462046FFF7ADFC32E0AFF30080EB
:1060D0008D49FD1A070000000054CE09F2AE000001
:1060E00040420F00005A62021D5500008D49FD1A02
:1060F000AD640000B1640000640B002000CA9A3B4C
:10610000B4F86230F31A190413D494F8583084F8B0
:10611000593004F11705052204F15D012846FBF70B
:10612000A2F905212846FCF718FE237F60F305033A
:10613000237794F8952094F894309A421DD0002249
:10614000114610460523FFF7CDF8D548FCF79FFD13
:10615000014690B194F8943084F89530037943F077
:106160000303037102234371C37194F896300372E1
:106170002046FFF757FC238E638694F8341094F87A
:106180002030C848A268039411F0010F03F10703FF
:10619000C549DBB208BF01468DE80C000291231D02
:1061A00022460A9940460136FFF7ACF866840DB0E6
:1061B000BDE8F08FBA48FCF76AFD07460028B8D062
:1061C00094F8349094F8583084F8593019F0010953
:1061D00045D104F1A5052B464A4604F1770104F1A7
:1061E0006700FCF733FE2946102204F1C600FBF7D6
:1061F0003AF904F1BE01082204F1DF00FBF733F99C
:1062000094F8BD3084F8B59069F3000384F8BD308C
:1062100094F8DE3084F8B69043F0010384F8DE3061
:1062200094F8A43084F8B79043F0300384F8B89021
:1062300084F8B99084F8BA9084F8BB9084F8BC9044
:10624000A4F8D690A4F8D890A4F8DA90A4F8DC903A
:1062500084F8A430391D2046FFF71EFCEBE494F8C7
:10626000A43003F04803082B00F08780037943F043
:106270000303037194F85C5045B1022343710D236D
:10628000C3710023057284F85C30D4E48448FCF7C1
:10629000FEFC814600283FF427AD037943F0030359
:1062A00003710D2343714FF0040A00F1080309F153
:1062B000100B80F807A008221846AA210B93FBF7C1
:1062C000FEF85246BB215846FBF7F9F80B9B082213
:1062D000194604F17F00FBF7C6F85246594604F10F
:1062E000C200FBF7C0F84946204604F1A509FFF7B4
:1062F00099FB4B462A4604F1770104F16700FCF74D
:10630000A5FD1022494604F1C600FBF7ACF80822AF
:1063100004F1BE0104F1DF00FBF7A5F894F8BD30ED
:1063200084F8B55043F0010384F8BD3094F8DE30B2
:1063300084F8B65065F3000384F8DE3094F8A43096
:1063400084F8B75043F0100384F8A430012384F894
:10635000B85084F8B95084F8BA5084F8BB5084F827
:10636000BC50A4F8D650A4F8D850A4F8DA50A4F839
:10637000DC507B710523FB715DE4D5F8200290F8B9
:10638000A43043F0200380F8A4300021FFF784FB01
:10639000D5F8202292F8A43003F0FB036FF3C30377
:1063A00082F8A43047E43E48FCF771FC054600281B
:1063B0003FF4BFAE94F8583084F859300F23C4F836
:1063C0008830037943F0030303710923437194F880
:1063D000343013F0010F0CBF08230E230822C371C1
:1063E00000211044FBF76BF8D4F888302B721A0A9E
:1063F0001B0C6A72AB7229462046FFF713FB238EF3
:10640000638696E694F88C30DA0721D42448FCF7AA
:106410003EFC014600283FF48CAE94F8583084F8D6
:10642000593094F88C3043F0010384F88C300379B0
:1064300043F003030371062343710C23C371092343
:1064400003724FF0FF3343728372C3720373D3E757
:106450009B077FF549AC94F8583084F859300220F6
:10646000FDF78AFF00283FF43FAC238CC380012353
:106470000371037A43F003030372062343720C2370
:10648000C37294F88D300373B4F88E30A0F80D30D9
:10649000B4F89030A0F80F30FEF7F0FC49E600BFEA
:1064A000640B00202558000011590000FFF72CBB99
:1064B000FFF72ABB0000000030B58DB0022309931E
:1064C000FF238DF8233009AB02937B4B01930AAB7A
:1064D000009304460BAB00200DF1230201210A902A
:1064E000FDF75AFE02280BD0099B6BB1404080F3A8
:1064F00011884FF0040002DF01210020FDF7C0FEEB
:10650000099B022BF8D0EFE79DF82330FF2B6B4B54
:1065100000F0AC800A9AA82A00F2A8801A783AB94A
:10652000012018701146664BFCF7AAFA0028DDD14D
:106530009DF82320042A65D9062AE4B264D9614B68
:10654000073A92B2FC21D3F81402FCF7CFFB0546C0
:1065500083684168994238BF19460368002B5BDAAB
:106560000A9A23F000431144CB1A0A93062C49D906
:10657000544BE21FD3F8140292B2FC21FCF7B6FB95
:106580000368002B04460ADA0A9A816823F0004364
:106590001344426891422CBF5B1A9B1A0A938DB335
:1065A000A38CAA8C9A422DD1474892B2A2FB00013B
:1065B00040F2231303FB02113DA3D3E90023F9F7B3
:1065C00029FE0A9B20F07F40002298423AD302B174
:1065D0000A9394F8342012F0010F95F8342034D047
:1065E000D0070FD4E2683B329A420BD92046FDF720
:1065F000E3FE022806D195F88C30990702D528468B
:10660000FDF7DAFE0DB030BD304800F1E803052A91
:1066100018BF184600259BE79942A7D25B1A9BB288
:1066200006902B490591002002939DF823200490A9
:106630000390019000900121FDF732FD30F002033C
:1066400094D053E71B1A0122BFE7D207DAD5E268DC
:106650003B329A42D6D92846FDF7AEFE0228D1D168
:1066600094F88C309B07CDD52046C9E71B7813B131
:106670000120FEF755FB9DF82320531FDBB2F92BB9
:10668000C0D8062A0DD90F4B073A92B2FC21D3F895
:106690001402FCF72BFB9DF823200121FEF7A2FB3F
:1066A000B0E70A4800F1E803052A18BF1846F2E7E8
:1066B0008D49FD1A07000000F1420000E80D00209E
:1066C00070020020040900200054CE09C8090020EF
:1066D000F5420000000000002DE9F04F91B0FCF7FA
:1066E00091FCC5B23DB3FCF7A9FC5FFA80F9FCF759
:1066F00017FDC6B2FCF7BEFEC4B2FCF7A1FEC3B2E2
:106700000A93FCF7D9FCC7B2FCF766FCFCF71AFD4C
:10671000FCF7FCFCFCF79AFEFCF7C6FC5A48037C2D
:106720008246052B29D8DFE813F051006C000D00DC
:10673000A209A209A209FF232F462C462E46A946EC
:106740000A93E1E701230374FCF7CAFD044696208F
:10675000FCF706FDFCF788FC9AF80F30013BCB34C0
:10676000032B0AD8DFE803F002203535FCF770FC74
:10677000FCF710FCFCF740FC28B1404080F3118886
:106780004FF0040002DF9AF8D43013F0C00F05D0A8
:106790009AF8430010B13D49FCF72CFE2046FCF767
:1067A00045FDFCF78BFD11E09AF84522DAF84032FE
:1067B00053F822000830FCF7EDFBFCF71DFC002825
:1067C000DBD12046FCF732FDFCF75EFC11B0BDE8E2
:1067D000F08F9AF84522DAF84032DAF8200253F8BE
:1067E00022100831FEF7B8FAFCF706FC0028C4D1E5
:1067F0002046FCF71BFDFCF761FD0120FEF74CFC79
:10680000E4E72DB903238AF81030FCF7DBFBDDE762
:10681000C37B013B032BB0D8DFE813F00400A401D5
:1068200015041504B9F1000FECD0FCF711FC037846
:1068300003F00F03032B05462AD143780C2BE1D13B
:106840009AF8D430580602D50EB9002CDAD00323BA
:106850008AF81030FCF710FC9AF8A5319AF8A621B6
:106860009A4206D00133DBB2022B08BF00238AF81C
:10687000A5319AF8A501272303FB00A000F25710C9
:10688000FCF78EFBA2E700BF0409002048090020A6
:10689000052BB7D14378222BB4D19AF8D430DB0939
:1068A00002D00EB9002CADD09AF886322BB19AF8EE
:1068B00084329AF885229A42A4D1DAF8A831002BC2
:1068C000A0D00320FDF758FD064600289AD04FF0CF
:1068D000040B8AF810B0FCF775FBDAF8A841DAF877
:1068E00014120027FC222046CAF8A871FCF701FA0E
:1068F0000322208405F1120104F11400FAF7B3FD1C
:1069000004F1100318465A4604F1170805F10E0168
:106910000D93FAF7A8FD052205F11E014046FAF78E
:10692000A2FD05214046FCF718FA227F0D9B60F37B
:106930000502227795F82320C2F30402A277B5F866
:106940001880A4F82480E97EAA7E42EA0122E2842B
:1069500019465A4604F15000FAF785FDAA8B40F219
:10696000E24942F2107309FB08F85343B3FBF8F312
:10697000A385C14BB3FBF8F32386238CF380294610
:106980000123F772337311F8023B4FF0030BC3F38B
:106990008013737386F804B0062206F10E00FAF72E
:1069A00062FD2946062211F8083BC3F3C013337574
:1069B00006F11500FAF757FD9DF82830F3762B8B7A
:1069C000B3836B8BF383AB8B338495F82330C3F3A2
:1069D000421386F82230208CFEF77CF9FEF74EFA3F
:1069E00095F8232094F83430A449520962F3430304
:1069F00084F834309AF82C3231F8122031F8133000
:106A0000134408FB03F303F574239D4A03F23F2369
:106A1000B3FBF2F34FEA5802963AA363E2636A7D4E
:106A2000A76409FB02F2E264DAF8886266604FF05C
:106A300027092822A8EB030840F286334E45E2607E
:106A4000C4F80090A7604FF00502009339468D4BC3
:106A5000384638BF4E46FDF769FB40F28731FEF7F6
:106A60004DFD9AF8553109FB03A999F8073103F058
:106A70000F03012B06D100973B465A46394638464C
:106A8000FDF754FB94F820307F4F0733DBB20D93B2
:106A9000DAF80430A3EB060BFCF722FCA8FB07890D
:106AA00071A3D3E90023824649464046F9F7B2FB79
:106AB00040F2A3330893754B0793754B06940593E7
:106AC000E368744ACDE90A011E4420F07F400723A1
:106AD0000021434302FB0133A0FB0201B8EB00009D
:106AE0001944B6B24FF000044FF47A724FF000032D
:106AF00069EB010104960394F9F78CFB0A9B029061
:106B000023F07F430193E88A80B2013040F2E245EE
:106B10004FF0000141F10001A0FB05230AF1FF3A0B
:106B200012EB0A0205FB013343F10003A2FB07014C
:106B300007FB03114EA7D7E9006780194AA3D3E9E1
:106B400000237941F9F766FB0D9A20F07F40009011
:106B50005B4621460846FDF75BFA30F002037FF4FE
:106B60000CAE33E6B9F1000F00F0128290F8BC21B0
:106B7000C2F300121AB116B9002C00F00982DAF83B
:106B800040329AF8451253F82160DAF80C32F3B12A
:106B90009AF886322BB19AF884329AF88512994283
:106BA00015D1337A190779D0337A03F00F02012A0D
:106BB0000DD19AF8BC21DB09B3EBD21F00F0BA81EA
:106BC0009AF8BC31C3F301139D0700F1BD81337AFC
:106BD00013F00F0202D0062A40F0E6819AF8BC11A9
:106BE000CC0740F1D181DAF80C12002940F0CC81B9
:106BF0003846FEF7B5F9002840F0CA81FCF728FABC
:106C000003782549032262F303039AF8BC21D209D1
:106C100062F386130370337A0278C3F3801363F34D
:106C2000C7120C2304464370027006220230FAF7A2
:106C30001AFC062206F10A0104F10800FAF713FC17
:106C40009AF8BC3143F002038AF8BC312046022393
:106C50008AF81030FCF7A4F99620FCF781FAFCF7CB
:106C6000FBF99EE5AFF300808D49FD1A0700000097
:106C700000DC356BD8FFFFFF005A6202F2AE000065
:106C800040420F00FD54000000CA9A3B1D55000011
:106C9000B16400008D49FD1AC70A0020002A00F0E7
:106CA0003681FCF71DFBDAF8B83100F5FB74D648E5
:106CB0000722A3FB000102FB0311CFA3D3E90023AA
:106CC000F9F7A8FA84424FF0000580D20320FDF7BF
:106CD00053FB8146002800F05B814FF00408DAF88E
:106CE0000C428AF81080CAF80C52FCF7B1F902780D
:106CF000052161F303029AF8BC1102F0DF02C90911
:106D000061F386120270327A0178C2F38012831C1A
:106D1000074662F3C711222201704270BB490D93EE
:106D20001846062207F1080BFAF79DFB06F10A0147
:106D300006225846FAF797FB424604F1100107F184
:106D40000E00FAF790FB032204F1140107F1120080
:106D5000FAF789FB01237B75BAF80232DAF8106280
:106D600040F2E24202FB03F8002E40F0FA80FCF70A
:106D7000B7FABD7500F24B66FD75BAF802323B8377
:106D8000BAF804327B83BAF80632BB8304F11701E8
:106D9000052207F11E00FAF766FBA27F97F8233061
:106DA00062F3040387F823309AF82C2262F3471326
:106DB00087F82330FCF760F93846FCF7F1F8FCF768
:106DC0001BF9054600287FF4D8ACFCF777FADAF80F
:106DD0001412FC222046FBF78CFF0323208489F841
:106DE0000B5089F80C5089F804303B78A9F806005C
:106DF000C3F3C01389F80D305946062209F10E007D
:106E0000FAF731FB3B780D99DFF814B2C3F3801326
:106E1000062289F8143009F11500FAF724FB9DF8D1
:106E2000283089F81B30BAF80232A9F81C30BAF8B9
:106E30000432A9F81E30BAF80632A9F8203097F8C3
:106E40002330C3F3421389F82230208CFDF742FF30
:106E5000FEF714F8DAF88872DAF80832E3602723CC
:106E60009F426760236038BF1F464FF49463062239
:106E7000A560294600932846654BFDF757F940F277
:106E8000A141FEF72BFB2B460422294600952846FC
:106E9000FDF74CF9DAF80430A3EB070A94F8203038
:106EA00006940733DBB20A934FF497630893594B68
:106EB0000793594B0593E3680395A8FB0B891F447F
:106EC000BFB24FA3D3E90023404649460497F9F7E0
:106ED000A1F9104619464FF47A720023F9F79AF98E
:106EE00047A3D3E90023029049464046F9F792F9B7
:106EF00043A3D3E900230190A6FB0B01F9F78AF91C
:106F000020F07F40009053460A9A294622E69AF8DC
:106F1000BC21C3F38013C2F380129A427FF444AEC3
:106F2000062206F10A013D48FAF788FA00283FF4E4
:106F3000B8AE39E6062206F110013448FAF77EFAB7
:106F400000283FF4AEAE3BE696F90830002BBFF6C2
:106F50003EAE737D03F0C003402B7FF438AEA0E655
:106F60004644002EFCDBFCF7BBF900F24B60864286
:106F7000F6D3FCF7B5F9A6F24B63181A40F2E243D8
:106F8000B0FBF3F0F882F8E672B9737A002B52D1B5
:106F900003238AF81030FCF715F89AF8BC316FF328
:106FA00041038AF8BC3111E4012A0DD0337A03F091
:106FB0000B02022AE9D003F00F03042BE8D19AF860
:106FC000BC319907E1D4E3E79AF8BC21DB09B3EBC4
:106FD000D21F27D09AF8BC31C3F301139807E5D527
:106FE00096F90830002BE1DA737D03F0C003402BE3
:106FF000DCD1CAE7AFF3008000CA9A3B0000000072
:107000008D49FD1A070000008D49FD1AC70A0020AE
:10701000DD5400001D550000AD640000C10A0020D1
:1070200000CA9A3B062206F110019048FAF706FAC8
:107030000028AAD0CEE7DAF80C32002BA8D13846C7
:10704000FDF78EFFA4E790F8243290F84522013333
:1070500080F82432D0F8403253F822600123337193
:10706000B9F1000F00F0D2844FF00008D0F82042B0
:1070700080F8258294F8A430317A03F00102C1F33C
:107080008001914200F0FA8082F0010262F3000375
:1070900084F8A430DBB21A0600F1EC80D4F8E88062
:1070A00094F8F92008F1040087187D78002D75D038
:1070B000815C9B0601F003010AD5D4F8D620D4F8F0
:1070C000DA30013243F10003C4F8D620C4F8DA30D4
:1070D000032963D1FB78023B0B2B5FD8DFE803F079
:1070E0000645975E5E5E5E5E60695E9E03238AF87B
:1070F0001030FBF767FFFBF77FFF00287FF43DAB05
:107100003979DAF82002132908BF1621FDF78EFE1F
:107110000124DAF8203293F8F920154493F8F82086
:10712000EDB2AA4283F8F9501CD1D3F8E820D3F885
:10713000EC1000208A4283F8F80083F8F90077D138
:10714000B8F1000F0ED01168D3F8F020C3F8EC109E
:107150009142C3F8E81008BFC3F8EC004449404628
:10716000FBF7AFFD4FF000086BE0082207F10E01BE
:1071700004F17700FAF777F9DAF82002042207F130
:107180001601BE30FAF76FF9DAF8203293F8A4202E
:1071900042F0080283F8A4201A8E5A860024B8E729
:1071A00094F8A43043F0480384F8A430238E638617
:1071B000F4E79AF80F70FFB2042F28D198F8043042
:1071C00043F0030388F80430172388F805300323BD
:1071D00088F80730082204F15D010430FAF743F91A
:1071E00094F8653088F8103094F8663088F81130DB
:1071F0000822CC2108F11200FAF761F908F11A000F
:107200003A46DD21FAF75BF94FF00008C6E794F83B
:10721000A43043F0080384F8A430BFE794F8A43006
:1072200003F0FB036FF3C30384F8A4300023BEE72D
:10723000D3F8F0108A42126808BFC3F8F020C3F8F0
:10724000E820DCB1DAF82002FDF774FF0023CAF869
:107250002032B8F1000F3FF4B9AA0025DAF8203245
:107260004146188CFDF7F4FE50E100BFC70A00202C
:10727000640B002068F3C71384F8A430DAF82032D6
:10728000327A93F8A430C2F3C002C3F340039A42A7
:1072900040F0CE830320FDF76FF8002800F0C8838C
:1072A0009AF88632A3B3DAF85032DAF854229342CD
:1072B00005D19AF884229AF88512914228D0DAF8FA
:1072C0005422934200F0B4839AF884329AF88522CB
:1072D0009A4200F0AD839AF8843233B9DAF820325A
:1072E000BAF882221B8C9A4212D09AF8843203F0A8
:1072F000FF05002B00F09D839AF88432DAF8201203
:107300000AEB4303B3F87C220B8C9A4240F0908343
:10731000777A002F00F07581DAF8203293F8A470A4
:1073200017F0100705D0FCF741F800283FF425AA14
:107330000127DAF8203293F8A430DA0626D4DAF8F6
:10734000204294F8A43013F0040F337A39D113F0AB
:1073500003033FF412AA022B40F22C81F57A112D7F
:1073600000F24383DFE815F03200E20009010D016D
:10737000280140014F0136037601AB01C201CE0165
:10738000E601410276014A024D010203FCF72CF8A6
:107390000028D4D103238AF81030FBF713FEFBF743
:1073A0002BFE044600287FF4E8A93D21DAF82002EC
:1073B000FDF73CFDDAF82002FDF7BCFECAF82042DA
:1073C00047E703F00302032AE4D1C0E7B6F815103B
:1073D000638CCB1A1B0400F1DE8494F8593094F8C6
:1073E00058209A420BD094F85A20012A7FF4C5A95C
:1073F00094F8852002F00702052A7FF4BEA9DAF886
:107400008C2232B994F83420D5077FF5B6A9CAF892
:107410008C42327B84F88420B6F80D0040F2E242C0
:107420004243E267307CF27B42EA0022A4F85C200F
:10743000B07C727C42EA0022A4F85E20F27C307DAF
:10744000A4F8641042EA0022A4F8602094F8852091
:1074500002F0F8026FF3C40284F88520013B012298
:10746000002584F85A2084F859306586DAF820120D
:1074700091F8A43083F0020381F8A4305FB1D1F811
:10748000B520D1F8B930013243F10003C1F8B5207D
:10749000C1F8B9300027DAF820020FA990F8A4400B
:1074A000FDF710F99AF81030032B4FEAD41415D0D9
:1074B000002F40F0C082B9F1000F07D0337ADB060D
:1074C00004D40F9B5B78002B00F0B582DAF82032F1
:1074D00093F89730002B0CBF02230323032B8AF869
:1074E000103040F0BC829AF80F30042B40F0A58297
:1074F000DAF8203293F8A42064F3C71283F8A420AA
:10750000FBF760FDB8F1000F7FF4A8AE002D3FF44B
:107510005DA9DAF82032188CFDF7DCFBDAF82032AE
:107520001B8CF380FDF7AAFCFFF750B9B6F81130B9
:10753000628C9B1A180400F12E8494F8582094F859
:1075400059309A427FF419A9052206F10C0104F181
:107550005D00F9F788FF737CB27C43EA0223A4F84C
:107560006230022384F85A3094F859300025013BE8
:1075700084F85C5084F8593078E7337B84F897308E
:107580003FE0082206F1160104F17700F9F76BFFDE
:10759000DAF82002042206F11E01BE30F9F763FF7B
:1075A000DAF8203293F8A42042F0040283F8A420F1
:1075B0001A8E5A86012559E7082206F10C0104F1BA
:1075C0007F00F9F750FFDAF82002042206F11401D7
:1075D000C230F9F748FFDAF8202292F8A43043F0DD
:1075E000040382F8A4300CE094F8582094F8593041
:1075F00093427FF4C2A80322013B84F85A2084F806
:107600005930002532E79AF80F20D2B2032A18D158
:1076100094F8581094F859308B427FF4AEA8013B8F
:1076200084F85A2084F8593094F8A430590605D5C6
:107630006FF3861384F8A430062333710023638626
:10764000B8E794F8A43003F0FB036FF3C30384F8A6
:10765000A430E9E7337B727BC34843F07F4343F4B4
:107660007E0343F4435343F0100343EA0223B27B07
:1076700043EA0243D4F88820C2F310021340C4F84E
:107680008830FBF704FB054600283FF476A8037911
:1076900043F003030371082209234371C3710021DE
:1076A0001044F9F70CFFD4F888302B721A0A1B0C1F
:1076B0006A72AB7229462046FEF7B4F9A1E7337B24
:1076C000727B43F07F4343F47E0343F4435343F020
:1076D000100343EA0223B27B43EA0243D4F8882032
:1076E000C2F310021340C4F88830A7E72046FEF723
:1076F000F3F9DAF8202292F8A43043F044036FF350
:1077000004136EE79AF80F30042B0AD12046FEF7D7
:10771000E3F9DAF8203293F8A4206FF3041283F827
:10772000A420DAF8202292F8A43043F004036FF387
:10773000451356E7337B84F88D30B27B737B94F826
:107740008C5043EA0223A4F88E30F37B327C43EA68
:107750000223A4F8903094F88C3005F0030001283F
:107760004FF0000543F0020304BF6586054613F0A1
:10777000010B84F88C307FF479AE43F0010384F878
:107780008C307948FBF783FA014600283EF4F5AFC8
:10779000037943F003030371062343710C23C37180
:1077A000092303724FF0FF3343728372C372037372
:1077B0002046FEF737F994F8A43043F0800384F8AC
:1077C000A430FBF741FC037880F801B0012262F39A
:1077D0000103D4F8E8200370DBB21AB143F01003C0
:1077E000037043E662F30413FAE794F8A43003F05D
:1077F000FB036FF3C30384F8A4301FE794F8592008
:1078000094F85830934268D1DAF88C32002B40F06B
:107810009680DAF88C320BB9CAF88C42717B337BD4
:1078200043EA0123A4F85C30717C337C43EA0123F2
:10783000A4F85E30708AA4F86000337D84F862306A
:10784000B17D737D43EA0123A4F86430317EF37D7A
:1078500043EA0123A4F86630B17E737E43EA012334
:10786000A4F86830317FF37E43EA0123A4F86A303C
:10787000B17F737F43EA0123A4F86C3096F820109F
:10788000F37F43EA0123A4F86E3096F8221096F8AD
:10789000213043EA0123A4F87030E16D636A994214
:1078A00002F1FF3294F885300AD1A18DA58C4D43A9
:1078B0007D2169434FF47A7591FBF5F1884226D01A
:1078C000042161F302036FF3C403012584F88530BA
:1078D00084F85A5084F85920C8E594F83450DAF8FE
:1078E0008C3215F0010521D09C427EF446AF94F80D
:1078F0005A30012B7EF441AF94F8853003F0070332
:10790000591E012985D9052B7EF437AF81E7032065
:10791000002560F30203012165F3C40384F8841099
:10792000E56784F8853084F85A10D3E79C427EF4EA
:1079300024AF94F85A30012B7EF41FAF96E50A4825
:10794000FBF7A5F9014600283EF417AF037943F091
:1079500003030371032343711123C3710F230372C4
:1079600020234372A7E600BF640B002094F8583030
:1079700094F859209A423FF444AE84F8593094F870
:107980005A30012B7EF4F9AEDAF88C329C427EF448
:10799000F4AE0023CAF88C3294F834206386D20700
:1079A00044BFA26F626594F8852012F0180F7FF42F
:1079B00028AEF37205223271E28CA38CF281A28D83
:1079C000B3815A437D2353434FF47A7293FBF2F30E
:1079D0003382EFE594F8583094F859209A423FF4F6
:1079E0002DAE84F85930FEF7C8BEBF48FBF74FF9FB
:1079F000014600283EF4C1AE0379057243F003034B
:107A00000371022343710723C37154E690F82532B2
:107A100013B9022380F825329AF82572013FFFB28C
:107A20008AF825720025B7FA87F77F09A84632E55C
:107A300000252F462FE5032350E5FBF71DFB0F998B
:107A4000DAF820020B7890F8A42062F3C303C2F3A3
:107A5000400262F382030B70FDF79EF952E5962017
:107A6000FBF77EFBFBF7F8FAFBF728FCE7E7C27BA6
:107A7000042A3EF682AEDFE812F0860105004000DF
:107A800091009100032B0DD190F8D43013F0380FF2
:107A900008D0FDF7A1FA02238AF81030FBF78CFA20
:107AA000FEF77FBEFBF728FB9AF81030032B55D169
:107AB0009AF85531272202FB03A393F8073103F00C
:107AC0000F03012B4AD040F6E12300210693874B98
:107AD0000593049140F247130391029101910091A3
:107AE00005220846FCF7DCFA30F0020336D09AF89B
:107AF0000E30052B32D0FEF740BE032B21D1D0F83B
:107B0000403290F8452253F822000830FBF742FA41
:107B10009620FBF725FBFBF7A7FAFBF7B5FA9AF8D7
:107B2000BC3113F0300F05D09AF8430010B1704902
:107B3000FBF760FC01238AF81030FBF737FAFEF7F9
:107B400030BEFBF7D9FA9AF81030052B06D1002386
:107B50000093042219461846FCF7E8FA00248AF834
:107B60000F408AF810408AF80D40FBF757FB224679
:107B7000214620465F4BFAF783FF044600287EF437
:107B8000FCADDAF80000436821465B6898470122A3
:107B900011462046FAF74CFFFEF718BED0F8200237
:107BA0000028DBD09AF80F30032B0CD190F89710F7
:107BB00049B1FDF73BF9DAF82002FDF7BBFA0023E3
:107BC000CAF82032CAE7468D9AF824429AF80F3054
:107BD000751CADB2002C5CD0032B55D1FBF764FBB8
:107BE000DAF82072DFF810918346786C00F14808CB
:107BF000C3453BA3D3E900233FD8A0FB0901F8F715
:107C000009FB84B2A8EB0B0035A3D3E90023A0FB4A
:107C10000901F8F7FFFA82B200237B64FB64FB8C56
:107C20007B85D7F8E83033B15B7913B997F8F93031
:107C30000BB100237B85DAF820320021D985DAF8F0
:107C40002002C38DBBB19D4280F095805B1B9BB22F
:107C50000021062BC385418540F28F809AF80F30B2
:107C6000032B08D1002E40F08880016D4B0811F0E5
:107C7000010143D10365002143E0ABFB0901F8F7A3
:107C8000C9FA022284B2C7E7002280F835201446E0
:107C9000D1E7042B0BD190F8971041B1FDF7C6F84E
:107CA000DAF82002FDF746FACAF8204256E79AF8B9
:107CB0000F30042B0CD190F835304BB19D4205D2DA
:107CC0005B1B80F8353000221446B8E73E2170E790
:107CD000C48D002CF7D1838DC3852246AFE700BF4A
:107CE0008D49FD1A07000000640B0020C5540000F8
:107CF000480900201002002000CA9A3B43F00043CC
:107D00000365438E1BB19D4239D25D1B458690F8B9
:107D1000595090F858309D4206D090F85A30013BA7
:107D2000012B9CBF0023438511B9438DB34228D05A
:107D3000438D01339BB224B91AB913B900293FF41A
:107D40000DAF90F820501548049107350021EDB291
:107D500005900393009223460695029101912A46CD
:107D60000846FCF79DF930F002033FF4F7AE9AF8AD
:107D70000E309D42BEE608211BE70121C1E722210A
:107D800017E70B46D7E7043B012B3EF6F6AC002382
:107D90000374FEF71BBD2823FFF7F0BBAD540000B2
:107DA0002DE9F041394D9DF818C0099CBDF82860B7
:107DB0002860C2EB821003F1030E85F82C12C5F87F
:107DC0001442A119043304EB80040CF10200BDF845
:107DD0001C80C5F84042DBB2C0B204EB83040CF156
:107DE00001074FEAC00C85F87802C5F8704204EB31
:107DF0000C0008F10304282C5FFA8EFEA5F83882E7
:107E000088BF08F10E0885F858E28BBF28F00308F8
:107E10000EEB4E0E18FB0EFE4FEA0E1EA5F83AE2D0
:107E2000B5F83A42C5F874024FF0300E6044A5F838
:107E30003CE2C5F83002B4FBFEFE20449C18C5F8B5
:107E4000480200EBC400BDF82040C5F85C020A34CB
:107E500024F003044830A4B2FFB2A5F86C4207FB3B
:107E60000404641A85F81C2285F8443285F83EE241
:107E7000C5F8640203D034442046BDE8F0810123F4
:107E800085F88632FDF7C0FBF6E700BF0409002045
:107E900038B503210520FCF73BFB04210620FCF745
:107EA00037FB1A4C002594F81C22ABB29A4205F11C
:107EB000010525D83021B4F83A22B2FBF1F284F85A
:107EC0003E2294F84422A4F83C120023013A84F89C
:107ED0004532637484F8793284F84330C4F8A831A9
:107EE000C4F80C3284F8463284F8582284F87A3286
:107EF00084F87B3284F87C32BDE83840FDF784BBDF
:107F0000A81DFF21C0B2FCF703FBCCE70409002049
:107F1000004870470B0A0020004870475B0A0020A9
:107F2000024B00225A749A74704700BF0409002063
:107F300070B5104B5E7CFF2E1AD00022D5B246FAE7
:107F400005F414F0010402F10102F7D10122AA4064
:107F500032435A7400F00102987CAA4002439A749A
:107F6000062202FB05301330F9F77DFA204670BD7A
:107F7000012070BD040900202DE9F843174C637CF3
:107F800006460F4643B108254FF006084FF0130987
:107F90006B1EDDB2FF2D02D10120BDE8F883637CAA
:107FA000EB40DA07F4D5A37C2B417340DB07EFD419
:107FB00018FB0590062239462044F9F73FFA0028BD
:107FC000E6D10123AB40627CDB43DBB21A40627432
:107FD000A27C1340A374BDE8F88300BF040900200D
:107FE0002DE9F04FDFF878B28FB0022391469BF86D
:107FF00056210D934FF0270840F2071318FB023863
:1080000007461BF8083003F00F03012B8A465E4633
:1080100000F2D680DBF8A8510DB10120CDE00BF5C0
:108020001370FAF734FE0B900028F6D00BF50670AB
:10803000FAF72DFE0B9A044628B90BF5137110467A
:10804000FAF73FFEE9E74FF6FF7303840F23C0F80A
:108050008830037FC57765F38613037790F8343053
:10806000458443F0010365F3041380F8343006239C
:10807000C38590F88C30058565F3000365F34103F3
:1080800080F88C3090F8A430458565F3000365F3E3
:10809000410365F3820365F3C30365F3041365F3DA
:1080A000451365F3861365F3C71305644564456599
:1080B000458680F8585080F8595080F8945080F8E0
:1080C000955080F89750C0F8982080F8A430C0F8F8
:1080D000E850C0F8EC50C0F8F050C0F8F45080F808
:1080E000F85080F8F950CBF8A80196F8D4306AF32C
:1080F000020369F3871386F8D430B9F1000F0BD06F
:108100005149B37C86F8D630302201F1C400F9F72A
:10811000AAF9737C86F8D530D6F88832C6F8C8300C
:10812000272B38BF272399461BF80830474DDFF827
:1081300034A12722C6F8C42003F00F030022C6F89A
:10814000CC20012B4FF08202C6F8D0200DF1340B69
:1081500049D1002F47D1FCF7A5F8D6F8D030CDF89B
:1081600020B04B449AB2049201938046034607958F
:108170000697CDF814A003970297009705220321D4
:108180003846FBF745FF02281ED00D9800BB304B48
:10819000059303224AF2FE330093CDF820B00795F1
:1081A0000690049003900290019043461146FBF71D
:1081B0002FFF02283ED00D9850B90FB0BDE8F08FC8
:1081C000002492E7FCF790F80D9B022BFAD0DCE735
:1081D000002C3FF422AF1F49D4F89800FAF771FD44
:1081E0001D4920462CE7FCF75DF807950025CDF8E2
:1081F00020B00695CDF814A0D6F8D030039580466F
:10820000994416480295BAB21FFA89F3A2FB0001FD
:108210000493912303FB021109A3D3E90023F7F789
:10822000F9FF009501904346052203212846BEE749
:10823000FCF75AF80D9B022BFAD0BCE7AFF3008095
:108240008D49FD1A0700000017090020F1420000C7
:10825000DD4E0000500B00201C0B0020002AE7849C
:10826000040900207D54000070B503210520FCF7AF
:108270004FF9054680B9094CD4F8A86166B1C4F835
:10828000A80104F51371D6F89800FAF71AFD04F561
:1082900006713046FAF715FD284670BD0409002026
:1082A00008B5FCF71FF968B190F8582090F85930DC
:1082B000934207D10133052280F8583080F85A20C4
:1082C000002008BD012008BD10B50C46FCF70AF9D6
:1082D00060B190F8952090F89430934206D1013324
:1082E00080F8964080F89430002010BD012010BD29
:1082F0002DE9F341054608461849D1F85032D1F826
:10830000542293420F461FD0D3F8048001F27B2100
:1083100098F80020FCF79CF80446E0B902AE97F804
:108320007B3206F8033D97F87C2231460DF10600BA
:10833000FCF78EF834B928B9C5F80080204602B0A1
:10834000BDE8F0810446EEE791F87C2201F27B2142
:10835000FCF77EF8044600232B60EFE704090020B9
:1083600013B5174C02AA002342F8043DD4F8540276
:1083700004F51471FAF7E4FC28B9404080F3118841
:108380004FF0040002DF04F51371FAF79AFC019B29
:108390001A79072AF1D80123934013F0EE0F03D185
:1083A000DB06EAD502B010BD94F8442294F85832A6
:1083B000013A9342E1DA013384F85832F2E700BF20
:1083C000040900202DE9F041154C05460068A4F58C
:1083D0000D76A4F11C0720B92860BDE8F041FDF737
:1083E000C9B80279D0F80080072A06D80123934043
:1083F00013F0EE0F07D1DB060AD4404080F311885A
:108400004FF0040002DF2146FAF75BFC4046E2E74A
:10841000C288D6F81402FC21FAF768FC3946F3E763
:10842000380B0020914210B5144B19D1D3F85422C7
:10843000D3F85042944211D1002914BF0A460322B6
:10844000013AD2B203EB420483F8852293F88422E6
:10845000A4F87E0291420FD083F88512012010BD4E
:1084600029B9B3F88232181A18BF012010BD03EBE6
:108470004103B3F87C32F6E7002010BD0409002068
:1084800030B4144B93F886220D4602B393F884223D
:10849000D1B293F8852235B14FF6FF73984216D0CA
:1084A00030BCFFF7BFBFD3F85002D3F85442A0420C
:1084B0000DD191420BD0D3F8544283F88512A042DB
:1084C00005D093F88402814208BF83F885220020FA
:1084D00030BC70470409002038B50B4CD4F840215B
:1084E000D4F8445122B10020C4F84001FBF782FDCA
:1084F0002DB10023C4F844310120FBF77BFD00209F
:10850000BDE83840FAF70ABB00B000400120FAF796
:1085100005BBFBF711B8684620F007018D4601B591
:10852000FAF7B6FC01F0D8F800F0D2FEBDE8014041
:1085300085467047012905D0404080F311884FF0EF
:10854000040002DF18200AB101F082B801F08EB8F1
:1085500011B90B2001F098B8012901D11820F9E7D1
:10856000404080F311884FF0040002DF88420AD0B7
:1085700018B94B1E584258417047012805D1B1FA2D
:1085800081F04009704701207047002070470000CB
:10859000084B39B101290AD0404080F311884FF0CF
:1085A000040002DF4FF40062C3F8002170474FF06F
:1085B0008072F9E700E100E070470000014B1868A5
:1085C00002F026B85811002070B5324B86B0186002
:1085D00008213148FAF760FF304801F011FA18B964
:1085E0006FF0120006B070BD436801211B68984708
:1085F000FAF7C4FBFAF7F2F9294B08221A700322A2
:108600001A720024274A1C7402260D251E760721A3
:1086100002928DE82800244A04232046FBF798FCA8
:10862000224801F0EDF90028DAD04FF4F8730493F2
:108630001F4B03931B2302930193224600960123B1
:108640000721FFF7ADFB044608BB024601460120A7
:1086500001F028F8224621460B2001F023F822469B
:108660002146182001F01EF822460121284601F07B
:1086700019F8012000F0ECFF0B2000F0E9FF1820B2
:1086800000F0E6FF284600F0E3FF2046AAE76FF07F
:108690000B00A7E758110020F80D00200AAD0000DC
:1086A00038110020FC0E0020000E002015AD000047
:1086B000940B002008B50B4638B121B106220749BA
:1086C0001846F8F7D0FE054808BD21B10622044936
:1086D0001846F8F7C8FE024808BD00BFEF0D00209D
:1086E000E90D0020062210B10248F8F7BCBE02488E
:1086F000FBE700BFEF0D0020E90D00202DE9F3415D
:1087000006248DF8024002248DF803400D463E4CAD
:1087100001211F4600238D428DF801108DF80410B1
:108720008DF800309DF8241008BF2380E37818BF2F
:10873000208061F30203E370A1789DF8283063F391
:10874000871102AB1D4415F8083C63F3030162F383
:1087500004110A466FF34512A270FFF7D9FB90F897
:108760004F5005EB8503C5EBC305A378425D63F36A
:10877000030202F0CF02C3F3001363F386124255E3
:10878000A27802F00F03012B064600EB050835D155
:1087900067F34512A27008991C480622F8F763FE99
:1087A0000622089908F10800F8F75DFE0C2388F806
:1087B0000130A378725DC3F3401363F3C71272559F
:1087C000FFF7AAFB90F84F2002EB8203C2EBC30233
:1087D0000421835C61F30303A17803F0CF03C1F3A9
:1087E000001161F386136FF3C713851883546B78F8
:1087F0000BB906236B7002B0BDE8F08198F8013028
:10880000002BD6D10623D2E75C1100206611002090
:108810002DE9F84307468846FFF77AFB90F84F406A
:1088200090F84E30A342054604D10134E4B2022C44
:1088300008BF002404EB8402C4EBC202DFF8689096
:10884000AB5C99F8021061F3030303F0CF03C1F3AB
:10885000001161F3861399F80210C1F3401161F31E
:10886000C713AE18AB5409F104010622B01CF8F787
:10887000FAFD99F8023003F00F03012B06F108000E
:108880000AD1062209F10A01F8F7EDFD0C237370F5
:1088900085F84F40BDE8F8833A4641460637F8F779
:1088A000E2FD7770F4E700BF5C1100202DE9F04194
:1088B00006460F46FFF730FB90F84F4090F84E30D9
:1088C000A342054604D10134E4B2022C08BF0024BF
:1088D00004EB8402C4EBC2020421AB5C61F303032A
:1088E0000F49887803F0CF03C0F3001060F38613BC
:1088F00005EB02086FF3C713AB54B31D88F80130C2
:108900000622043108F10200F8F7ADFD324639467F
:1089100008F10800F8F7A7FD85F84F40BDE8F081A1
:108920005C11002070B518B9BDE87040FFF79CBC21
:10893000FFF7EEFA0646FFF7EFFA96F84F20134CD2
:1089400002EB8203C2EBC30290F84F30164403EBF4
:108950008302C3EBC203C518A078211DC0F3001029
:10896000FFF7A8FE211D0622B01CF8F77CFD211D93
:108970000622A81CF8F777FDA278E17820889209F2
:1089800001F00701BDE87040FFF72ABB5C11002031
:1089900070B504464FF02003EFF3118583F311887F
:1089A000438B4BB3028B9A420FD9002101F00EFC8E
:1089B00058B185F3118801230371002343710360CB
:1089C000038200F11403C3601CE0668B731E638393
:1089D00085F31188A18BE08B238B0330CA1C22F016
:1089E000030220F003001044626A14309B1B03FB57
:1089F000002084604182DEE785F3118801F0E6FB08
:108A00000028D8D170BD00F114031944C16070472B
:108A100010B40A46146814B910BC01F091BB537924
:108A200043F0010353712246F4E710B5014601B942
:108A300010BD0B790C68013BDBB20B71002BF7D139
:108A400088680B60036A1BB1084698472146EEE729
:108A500001F072FBFAE703790133037170478388F1
:108A6000026819448180D018704730B48388046844
:108A70009D188580E01830BCF8F7F5BC83885B1A38
:108A800083800368194401600846704708B503688D
:108A900001211A78FFF7F2FF104608BD00F1080324
:108AA0000068C01A7047000008B5024800F0D6FA06
:108AB000002008BD02AF0000F8B50B4E0B4DAD1BFA
:108AC0000746ED100024AC4203DB4FF0FF34204694
:108AD000F8BD142256F834103846F8F793FC0028F5
:108AE000F5D00134EFE700BF08040020180400208F
:108AF00038B50546F8F771FC142807D929460F4800
:108B0000F8F78AFE4FF0FF34204638BD2846FFF7BD
:108B1000D3FF431C044604D129460948F8F77CFEDC
:108B2000F2E7084B1422186029460748F8F735FC8D
:108B300006490548F8F777FC0024E5E758AF000040
:108B40008CAF0000C00200203013002007AF0000EF
:108B5000012808B505D1054B4FF0FF321A600020FF
:108B600008BD4868FFF7C4FFF9E700BFC002002056
:108B700008B5084B1B6833B9074B1B68013306D196
:108B8000064B186808BD98470028F5D008BD044872
:108B9000FCE700BF70110020C00200204813002035
:108BA0003013002070B504684FF0FF3305460E46C1
:108BB0000B6024B90F48F8F72FFE204670BD0E4B0E
:108BC0001B685A1C14D143680BB11B782BB90B4896
:108BD0002146F8F721FE002070BD2046FFF76CFF0C
:108BE0003060013002D129680548F2E7686870BD3D
:108BF0000B60E2E715AF0000C00200202BAF0000C1
:108C000045AF00002DE9F04F442989B080460F465A
:108C100001D9002076E0002343540446234613F88C
:108C2000012B202A19D0002AF3D0DFF87CA12021C3
:108C30002046DAF80060F8F7C1FBDAF80030B6F148
:108C4000FF3F14BFA1464FF000090133054606D08F
:108C50000028DED1731C1FD1DBE71C46DEE70028AD
:108C6000D7D0061B721C132AD3DC214603A8F8F7C1
:108C700094FB08AB1E4403A8002306F8143CFFF73E
:108C80001BFF421C0646C4D005F1010920214846BD
:108C9000F8F794FB0028BCD14846F8F79EFBF30098
:108CA0000193019A3B4B00904FF0000A4FF0FF34C4
:108CB000554603EB020BDBF8042052F80A6026BB92
:108CC000002DA6D0002C52DBFFF752FF01463248A0
:108CD000F8F7A2FD41463048F8F79EFD009BDFF80B
:108CE000CCB005EB0309A9EB05039C4245DC2EB192
:108CF0002A48F8F791FD202308F80730009BA019B7
:108D0000C01AC0B209B0BDE8F08F3146009A48469B
:108D1000F8F778FB064620B935B9DBF8042052F89D
:108D20000A500AF10C0AC6E7002C07DA29461C484B
:108D3000F8F772FD2846F8F750FB0446154B019AE8
:108D40009A18A64206DA5168A85D51F80A10895DA2
:108D500088420AD00F4B019A12489A18344652683A
:108D600052F80A10F8F758FDDBE70136E9E7284624
:108D7000F8F733FB01260446B0E799F8001058468F
:108D8000F8F74AFD7B1C19F8012B08F80720DFB221
:108D9000A9E700BF080400200FAF00007EB5000067
:108DA0000AAF00000BAF0000C002002012AF0000AD
:108DB000F7B502A94FF0FF3341F8043D0746FFF72E
:108DC000F1FE019B5A1C06461DD0E0B1104D002457
:108DD00005EBC3056B68195921B939680D48F8F7D7
:108DE0001BFD10E03046F8F700FB04F10C0368B9F6
:108DF0006B68094909481A199268002A08BF0A468F
:108E00001959F8F709FD002003B0F0BD1C46E1E751
:108E1000080400202BAF00005EAE000034B000005C
:108E20000228F8B50D4605DC204B1C68621C06D0F4
:108E3000022815D1281DBDE8F840FFF7B9BF022868
:108E400020D01B481B4E1C4C1C4FF8F7E5FCA41B04
:108E5000E4100025A54221DB1948F8F7DDFC1BE0F2
:108E60000128EED11748154EF8F7D6FC114B002516
:108E700003EBC404636859590C3569B13046F8F7FF
:108E8000CBFCF7E74868FFF717FE431C0446E9D11F
:108E900069680D48F8F7C0FC0020F8BD56F8351099
:108EA0003846F8F7B9FC0135D4E700BFC00200200E
:108EB00041B0000008040020180400200BAF00009F
:108EC00055B000003BB0000045AF00002DE9F04F69
:108ED000534FDFF88481534E8DB0FFF749FE0146B2
:108EE0003846F8F799FC4FF0FF31404601F06EF933
:108EF000041D05462046F8F770FA002841D0237873
:108F0000202B204604F10104F9D0002B39D00DF1BB
:108F10003009012449F82C0D4FF0000A2021F8F700
:108F20004DFA40B1034603F801AB184613F8012B84
:108F3000202AFAD0E2B90CAB03EB8403002243F8F9
:108F40002C2CDDF804904FF0FF330093B9F1000FA3
:108F50001CD13548F8F760FC344B1B68002B4FD10F
:108F600001993348F8F758FC3248F8F755FC08E007
:108F700049F8240001340B2CD0D10A212E48F8F7EF
:108F80004BFC2946304601F0D3F8A6E799F80030AB
:108F9000002BDED029494846F8F727FA00283AD0B6
:108FA00027494846F8F721FA002836D0012C05D188
:108FB000244B1B68013301D12348CBE7694601A844
:108FC000FFF7F0FD009B5A1C8346C5D00028C3D094
:108FD0001E4A4FF0000902EBC30ADAF8043053F8D6
:108FE00009100029B8D05846F8F7FFF909F10C0329
:108FF00078B9DAF804309944D9F80430002BABD0B2
:1090000001A9204698470028BBDA01A8FFF7D0FE47
:10901000B7E79946E1E70E4BF2E70E4BF0E700BFEA
:109020000FAF000074110020D6AF00006C110020BB
:109030002BAF000008B00000B7AF0000E9AF0000A0
:10904000EEAF0000C0020020F5AF000008040020D1
:10905000218E0000518B00001813002010B504462B
:1090600086B0184801F00AF8174801F007F81749C8
:10907000154801F05DF81649134801F059F81549F3
:10908000114801F055F8144B14491548002C08BF3D
:109090001C46144B6FF008021C60002305930493D8
:1090A00003920293019300934FF4FA620E4B01F086
:1090B000C3FC0E4A0349044806B0BDE81040F7F768
:1090C000ABBC00BF18130020741100208C110020CD
:1090D00010120020941200205EAE0000981B0020A9
:1090E0004C13002048130020CD8E0000058C00009A
:1090F00008B500F0E9FC002008BD00002DE9F743A9
:109100001048114D114E124FF8F786FB114BD3F852
:1091100020411CB9204603B0BDE8F08301F0CAF934
:1091200084420CBFA846B046204694F8089001F04F
:1091300077F9224600904B4641463846F8F76CFBDB
:10914000A46DE6E7A1B000009FB000007EB500006E
:10915000A9B00000A014002008B5F7F767FE01468B
:109160000248F8F759FB002008BD00BF89B0000095
:1091700008B501F0AFFA01460248F8F74DFB0020B0
:1091800008BD00BFCDB0000008B5F8F7F9F8C0F38E
:109190000723C0F30742010E0248F8F73DFB002009
:1091A00008BD00BFDCB000000C4B1B78062B12D1B1
:1091B0000B4B186810F00F000DD104331B6803F03F
:1091C000F003302B08D1074B1B6813F0F00F0CBFD6
:1091D0000120002070470020704700BFE00F00F022
:1091E000E40F00F0EC0F00F008B54FF02003EFF3B0
:1091F000118183F31188FFF7D7FF20B12D4AD3687F
:1092000023F08073D360FFF7CFFF10B12A4B032206
:109210001A60FFF7C9FF30B14FF080430022C3F856
:109220000C21C3F810214FF01023D3F80022002A9C
:1092300003DBD3F80032002B2FDA204B0122C3F8D6
:109240000425D3F80024002AFBD04FF0102215216A
:10925000C2F80012D3F80024002AFBD04FF01023EC
:109260001522C3F80422154B1A46D3F8001400291E
:10927000FBD00021C3F80415D2F80034002BFBD03A
:10928000BFF34F8F0E490F4BCA6802F4E0621343DD
:10929000CB60BFF34F8F00BFFDE7094B4FF0FF32AC
:1092A0009A62DA62084B094A1A6081F31188002039
:1092B00008BD00BFF0ED00E0A005004000E0014067
:1092C00000ED00E00400FA050C0300200090D0033C
:1092D00000B501F019F95DF804EB00BF064881689C
:1092E0004A897F2A06D88069884203D003494FF013
:1092F00080520A6070470000A014002004ED00E0D6
:10930000044800232021C2180133272B82F80013C0
:10931000F9D1704700E100E00E498A682820104426
:10932000EFF3098C80E8F01F0B4F4FF00066202010
:1093300080F311888A698A603E60906E002393668C
:1093400080F3118802F1280090E8F01F8CF309885F
:1093500070470000A014002004ED00E01EF0040F90
:109360000CBFEFF30880EFF30980816931F8021C2C
:1093700011F0FF0101D0022907D0404080F311888D
:1093800004494FF080520A60704700B500F046FA79
:1093900000BD000004ED00E004498A6890660449BD
:1093A0000968D16600DFD06E70470000A01400206D
:1093B00054B5000010B5044601F07CF8226801465F
:1093C000BDE810400148F8F727BA00BF5AB20000C4
:1093D00010B504461A48F8F71FFA04F11800194CA2
:1093E000FFF7E8FFA36A9A0102D51748F8F714FAC5
:1093F000A36ADB0102D51548F8F70EFAA36A180331
:1094000002D51348F8F708FA0E4CA36A590302D59F
:109410001048F8F701FAA36A9A0302D50E48F8F744
:10942000FBF9A36ADB0302D50C48F8F7F5F9054A06
:10943000936A6FEA03436FEA1343936210BD00BF60
:109440002BB3000000ED00E044B3000058B300006F
:1094500073B3000092B30000B8B30000D3B30000B0
:1094600038B5044617480D46F8F7D6F904F1180048
:10947000154CFFF79FFFA36ADB0604D51348BDE830
:109480003840F8F7C9B9A36A180701D51048F6E7BC
:10949000A36A99070FD50F48F8F7BEF9A36A1A0611
:1094A0000ED5616B0C48F8F7B7F94DB1A36A23F0FC
:1094B0008003A36238BDA36ADB0701D50748DEE756
:1094C00038BD00BFA4B2000000ED00E0BBB2000058
:1094D000CDB20000E1B20000FAB200000BB3000010
:1094E00038B504461B480D46F8F796F904F1180004
:1094F000194CFFF75FFFA36AD90404D51748BDE8EC
:109500003840F8F789B9A36A1A0501D51448F6E777
:10951000A36A9B0514D51348F8F77EF9A36A1804CB
:1095200008D5A16B1048F8F777F91DB1A36A23F4A9
:109530000043A362084B9B6A590509D50B48DEE737
:10954000A36A5A05FAD4A36ADB0501D50848D6E711
:1095500038BD00BF21B1000000ED00E0BBB200004B
:10956000CDB2000038B10000FAB2000052B10000E4
:109570006EB1000038B5274D6B68C3F30803DA1EDF
:109580000446092A3AD8DFE802F00533352F393985
:10959000393939372048F8F73FF9EB6A9A0703D58C
:1095A0001E48F8F739F90CE0EB6A5B0009D51C4856
:1095B000F8F732F91B4B1B784BB101212046FFF71E
:1095C0004FFF21460020BDE8384000F02BB9164B74
:1095D0001B7823B101212046FFF782FFF1E7134BEF
:1095E0001B889BB2002BECD02046FFF7F1FEE8E78A
:1095F0000021E3E70021EEE70D48D2E70D480E49D0
:10960000A3F110020F2BD8BF01460C48F8F704F95C
:10961000D7E700BF00ED00E0B5B10000CDB100001C
:10962000EFB1000028ED00E029ED00E02CED00E0B6
:109630000FB2000087B100009CB1000046B20000EC
:10964000024A536943F010035361704700ED00E094
:1096500043B2012200F01F0002FA00F05B09024A47
:1096600042F82300704700BF00E100E043B201224E
:109670005B0900F01F0002FA00F02033014A42F8B3
:109680002300704700E100E04209054B00F01F0095
:1096900053F82220012303FA00F01040704700BF66
:1096A00000E100E043B2002BA8BF03F1604301F1E9
:1096B00001014FEA4111BBBF00F00F00044B03F55D
:1096C0006143C9B2AABFC9B2195483F800137047E5
:1096D00014ED00E000F05CB808B572B6044B5869B0
:1096E00018B100225A6100F0A5F962B608BD00BFAA
:1096F000A01400202DE9F0410F4604468D1838468D
:10970000AA2190461E46F7F7DAFE0A9B09992046E1
:10971000042201F01DFA1648276625F00702A2F17F
:109720002003002120F00100E1642165C4F8648079
:1097300042F8080C42F8206C069A5A60079A9A6020
:10974000089ADA604FF08072DA616365A364A166FB
:109750004FF02003EFF3118283F31188054BD3F808
:109760002011A165C3F8204182F31188BDE8F08182
:109770000DAA0000A0140020014910220A607047C1
:1097800010ED00E0404080F3118830BF704700BF0B
:10979000404080F31188DFF81CC0DCF800C01CF4E6
:1097A000006C0CBFEFF30880EFF3098000B5FFF702
:1097B000E1FE00BD04ED00E038B5431E04460D4651
:1097C000042B1AD8DFE803F00319131517000D480E
:1097D000F8F722F800F06EFEAA6901460A48F8F789
:1097E0001BF829462046BDE8384000F01BB8074862
:1097F000EEE70748ECE70748EAE701460648F8F7CE
:109800000BF8E7E7FFB30000A7B4000029B400009D
:109810004FB4000069B4000084B400000146006841
:10982000FFF7CABF052810B50CD001F0BDF860B134
:1098300001F0BAF80C4B0D49002808BF19460C4836
:10984000F7F7EAFFFFF79EFFFCE701F0BDF80028FD
:10985000EED1084C0848A168F7F7DEFFA068BDE824
:10986000104000F00BB800BFE7B40000E3B4000004
:10987000F8B40000A014002018B5000038B5054663
:109880004FF02003EFF3118483F3118801F0F0F817
:10989000284601F0A1F80B4B9B689D420DD10A4B65
:1098A0005A68C2F3080222B900F02EFE2046FFF7E4
:1098B00073FD5A6842F080525A602046BDE8384035
:1098C00000F084BDA014002000ED00E000B572B6E9
:1098D0000B4A506900281EBF0021516100F0AAF810
:1098E00062B6EFF30580A0F110004FEAC000054911
:1098F000014409C998475DF804EBFFF7E9BC000093
:10990000A0140020DC000000202080F3118808480B
:10991000AA214FF40062F7F7D2FD05484FF4006129
:10992000401880F30988022080F3148800F006B8FC
:10993000A42E002030BFFFF7FDBF00BF08B5074BC6
:10994000074A23F07F039360BFF34F8FBFF36F8FFE
:1099500000F0EAF800F0F2F800F010F90000000062
:1099600000ED00E008B5FFF7E5FFBDE80840FFF7B0
:10997000B5BC0000154B16491A6830B50D68C2F326
:10998000072295420FD8002248685A60954200F19C
:109990000C000AD105225A600E4B01221A70BFF347
:1099A0004F8FBFF36F8F002030BD50F80C1C50F864
:1099B000044C9A6021F01F0141F01001114344F062
:1099C0000104D96001321C61E0E700BF90ED00E0C6
:1099D00010030020BC13002038B5084B53F820407A
:1099E000013053F820502046A84204F10C0400D363
:1099F00038BD54F80C3C5B689847F4E740B500006C
:109A000070B50A4C0A4D0646AC4201D100240AE06A
:109A100063680BB90C34F7E7236830461968F7F729
:109A2000E4FC0028F6D1204670BD00BF6003002092
:109A300008040020431C03D0034B1B68984201DB41
:109A4000F7F7A2B9704700BF540300200F4D80B54F
:109A50000F4F05F10C064FF02002EFF3118382F354
:109A60001188EB68B3420AD04BB11C69631C08D063
:109A70003B68A34205DD6C61FFF784FEEBE74FF026
:109A8000FF342046F7F76CF9F5E700BFA01400207B
:109A9000540300201FB500239A4202D0CC5CAA2CAC
:109AA0000DD0D41A642161430192B1FBF2F100940C
:109AB000029101460348F7F7AFFE04B010BD013331
:109AC000EAE700BF2BAE000008B50E48F7F7A4FE8A
:109AD0004FF480620C490D48FFF7DCFF4FF4A07291
:109AE0000B490C48FFF7D6FF4FF400620A490B48B8
:109AF000FFF7D0FF4FF4806209490A48BDE80840EB
:109B0000FFF7C8BF5CB50000642900206CB50000F9
:109B1000642D002076B50000A42E002080B5000042
:109B2000A43600208AB500000248034A0021121A18
:109B3000F7F7C5BC60040020581700200248034A0C
:109B40000349121AF7F78FBC0000002060040020C0
:109B500094B5000008B50220FFF73EFF0320FFF791
:109B60003BFF00F0ABFFF6F713FD034A137A23F037
:109B70000103137208BD00BF3014002080B586B009
:109B8000324D06AFFFF7BCFB20235A195A51083358
:109B9000B3F5907F5260F8D12D4EDFF8DC80AE61D6
:109BA00000244FF0010943464FF480622949CDF863
:109BB000109030460394029401940094FFF79AFDAC
:109BC000737A304623F00403737200F04DFB0F23C9
:109BD00003932149CDF810900294019400941F4BF7
:109BE0001F484FF4A072FFF785FD1D4B1C4A5B7A9E
:109BF00023F004035372104600F036FB194BEB6060
:109C00002B61194B83F30888184BE02283F822203C
:109C1000DC771C765C769C765A6A42F4E0225A62C3
:109C2000FFF70EFDFFF7A8FD2046FFF7D5FE4846DB
:109C3000FFF7D2FE0E4BAE6023F007030D4A83F30D
:109C40000988002181F3118840461047A0140020A4
:109C50003014002064290020642D00204D9A00005B
:109C6000C0130020AC140020A436002000ED00E05A
:109C7000642D00200DAA0000559B000010B50A4B72
:109C80000A490B4A8B4201D3002010BD4FF020043B
:109C9000EFF3118084F3118814685C61136080F322
:109CA00011881833EEE700BF30040020480400207C
:109CB000B016002038B590F90A308B4204460D46A4
:109CC0000ED0437ADB060AD1036A013307D100F0D4
:109CD000F1FAA5722046BDE8384000F0C5BAA57279
:109CE00038BD000070B5304A0D469168CB7A013B13
:109CF0000446CB72C36811464BB1806892689042AB
:109D000011D095B900F07CFB6FF00F0070BD926828
:109D100092F90A2022610133E3608B68A36000F0AE
:109D20006FFB002070BD2269F4E792F90A1090F9E8
:109D30000A309942A8BF194621EAE1714FF0200389
:109D4000EFF3118683F31188A06890F90A309942E5
:109D500001DAFFF7AFFF2046294600F011FB00F0C3
:109D6000D3FB3046FFF718FB0028D8D023682169C1
:109D70009C4208BF002333B193F90A309942A8BF2F
:109D8000194621EAE1714FF02003EFF3118583F3C7
:109D90001188A068FFF78EFF85F3118800F030FB73
:109DA0006FF00A0070BD00BFA0140020F8B5344E5B
:109DB000B268D37A013B0546D372C368013BC360E6
:109DC0001BB1BDE8F84000F01BBB4FF02003EFF3E0
:109DD000118783F3118801698068FFF76BFF294BB6
:109DE0002C681B6883B1A54208BF002424B987F3FF
:109DF00011880023AB60E4E7236A023308D16B6863
:109E00009C42F4D02468F1E7A542F0D0002CEED0BB
:109E100094E80C001A6022685360637A216A23F088
:109E2000020363724B1C04F110020ED033699A4294
:109E30001FBF226913695B181361636922691A6085
:109E4000226953604FF0FF332362637A23F00402E8
:109E500013F01B0F627202D1236A01330BD087F318
:109E600011880023E366EB68AC600133EB6094F982
:109E70000A302B61A5E7204600F0F6F9EFE700BFB6
:109E8000A0140020C0160020F8B50023136003685A
:109E900007460E461546002B49D01868437A23F032
:109EA000200242729A0742D5036A02334BD090E8EF
:109EB0000C001A6002685360437A016A23F00203BF
:109EC00043724B1C00F110020FD0204B1B699A42C9
:109ED0001FBF026913695B181361436902691A6045
:109EE000026953604FF0FF3303620023C366437A75
:109EF00013F01F041BD1036A013318D100F0B4F929
:109F0000EFF305830D2B1CD823B1114B586810F4C7
:109F100000600BD00D4B9B685B897F2B01D9002023
:109F200004E000F03DFA003018BF012028607B6893
:109F3000C3F30432164366F3103300207B603860AD
:109F4000F8BD2046F2E76FF00A00F8BDA01400202B
:109F500000ED00E007B50346002200681A6001AA80
:109F6000FFF792FF019803B05DF804FB10B50A4BB0
:109F70000A490B4A8B4201D3002010BD4FF0200448
:109F8000EFF3118084F3118814685C61136080F32F
:109F900011881833EEE700BF480400206004002059
:109FA000B4160020427A22F0040112F01B0F417215
:109FB00004D1036A013301D100F056B97047036937
:109FC0001BB108211030FFF7C5BF1846704710B508
:109FD000044600F099FA2046BDE81040FFF7DCB9CE
:109FE00008B5064B9B685B897F2B05D800F0D8F934
:109FF000003018BF012008BD002008BDA0140020BB
:10A00000104A1268034600686AB1834208BF002004
:10A0100008B900207047026A023207D15A6890429C
:10A02000F7D00068F4E783420AD050B190E80C0002
:10A030001A6002685360437A23F002034372704748
:10A0400010467047C016002003695A1C11D00A4AF6
:10A05000126990421FBF01680A699B180B6190E862
:10A060000C001A60026853604FF0FF330361002058
:10A0700070471846704700BFA0140020002383607B
:10A08000C3600060406003614FF02003EFF3118272
:10A0900083F31188034B19684161186082F31188BA
:10A0A000704700BFB4160020F8B5054614464FF0BF
:10A0B0002003EFF3118783F31188FFF7A1FF064612
:10A0C000A0B11030FFF7C0FF3046FFF76BFF002351
:10A0D000F366F460EFF305830D2B23D81BB1134B0C
:10A0E0005B681B051ED5FFF77BFF11E031B9AB683C
:10A0F0002360EB68AC6043B9EC6006E00B6823605A
:10A1000073B9EB6853B9EC60AC602846FFF757FFB2
:10A1100040B13846BDE8F840FFF759BF1C60EBE797
:10A120000C60F2E787F31188F8BD00BF00ED00E096
:10A130000A46C168FFF7B8BF0A460021FFF7B4BF5F
:10A140002DE9F04704460D4691464FF02003EFF30A
:10A15000118883F3118807684FF0000AB84208BFDE
:10A1600000274DB12046FFF74BFF064688B9E3684C
:10A17000DBB9A560C4F80C90CFB1EFF305830D2BCC
:10A180001ED81BB1104B5B681B0519D5FFF728FFC4
:10A1900010E006F11000FFF757FF3046FFF702FF0F
:10A1A000F560C6F86CA02D68DBE71D60E2E720468D
:10A1B000FFF705FF20B14046BDE8F047FFF707BFB6
:10A1C00088F31188BDE8F08700ED00E038B54FF066
:10A1D0002004EFF3118584F3118884684CB1C168C1
:10A1E000226882608C4208BFC26085F311882046D5
:10A1F00038BD19B985F31188084638BD00F0C0F89C
:10A200002846FFF7E4FE0028F1D1024B9B68D8688E
:10A2100038BD00BFA014002030B5CA60114A886064
:10A2200010460B6150F80C3F83420CD10860136953
:10A230004B6013691960116130BD641B0C611469B6
:10A24000A342F3D01B68002BF0D00C691D69AC420F
:10A25000F3DC5A682C1B1C614A600B605A68116061
:10A26000596030BDA014002030B590F90A30104C70
:10A2700003F110014A11063204EB820201F01F05BE
:10A280000121A9405568143304EBC30329435160ED
:10A2900003605A6842605A6810605860A36990F978
:10A2A0000A1093F90A209142A8BF1846A06130BD58
:10A2B000A014002090E80A0010B590F90A20196057
:10A2C000016814324B60144B03EBC20153F8322087
:10A2D0008A420FD190F90A1010314A11063203EB6D
:10A2E0008202012401F01F0104FA01F1546824EAFA
:10A2F000010454609A6990420BD1D96991FAA1F294
:10A300000029B2FA82F208BF4FF0FF32043253F84C
:10A3100032209A6110BD00BFA014002030B40C6838
:10A32000A14208BF002434B901604B6843604B6808
:10A33000186048600BE090F90A5094F90A309D4289
:10A3400016DA636843600460636818606060437A8B
:10A3500043F002034372531C0FD009320A2330BC6E
:10A36000B2FBF3F30A46013300F11001FFF754BFCB
:10A370004B689C42D8D02468D5E730BC70470000B9
:10A3800070B5064C0E460546A068FFF793FF3246AF
:10A390002946A068BDE87040FFF7C0BFA0140020A8
:10A3A000094AD1699268002991FAA1F392F90A0049
:10A3B000B3FA83F308BF4FF0FF33103B9842D4BF8A
:10A3C00000200120704700BFA014002010B50A4BE8
:10A3D0009B685B897F2B044602D8FFF7E1FF10B929
:10A3E00084F3118810BD054B00222046BDE81040C3
:10A3F0001A60FEF7D1BF00BFA0140020C4160020D1
:10A400004FF02003EFF3118083F31188034B9A6818
:10A41000D37A0133D372FFF7D9BF00BFA014002055
:10A4200090F90A007047000010B590F90A30114AFF
:10A43000143302EBC303596888421AD04168046898
:10A440000C60046861600360596841605968086085
:10A450005860936998420BD1D16991FAA1F3002910
:10A46000B3FA83F308BF4FF0FF33043352F83330AD
:10A47000936110BDA014002038B54FF02003EFF316
:10A48000118583F31188094CA068FFF7CDFFA268FE
:10A49000A3699A4202D185F3118838BD044B00228A
:10A4A0001A602846BDE83840FEF776BFA0140020A9
:10A4B000C4160020014B9868704700BFA01400200C
:10A4C0000D4B1B68002B14DD0C4B1B68984210D001
:10A4D0000B4A90F90A30126893420ADB094A143396
:10A4E00002EBC30152F833004B68C01A18BF0120B9
:10A4F00070470020704700BFC415002058B5000009
:10A50000C8150020A0140020014B00221A607047DB
:10A51000C416002010B50A4B0A490B4A8B4201D3DE
:10A52000002010BD4FF02004EFF3118084F3118858
:10A5300014685C61136080F311881833EEE700BF84
:10A540001804002030040020B8160020427A22F0BF
:10A55000040112F01B0F417204D1036A013301D1CF
:10A56000FFF782BE70470000104A12680346006879
:10A570006AB1834208BF002008B900207047026A10
:10A58000023207D15A689042F7D00068F4E783425C
:10A590000AD050B190E80C001A6002685360437A08
:10A5A00023F002034372704710467047C016002024
:10A5B00003695A1C11D00A4A126990421FBF0168F0
:10A5C0000A699B180B6190E80C001A6002685360DE
:10A5D0004FF0FF330361002070471846704700BFFB
:10A5E000A014002000238160C2600060406003610D
:10A5F0004FF02003EFF3118283F31188034B1968A6
:10A600004161186082F31188704700BFB8160020BE
:10A6100070B504464FF02003EFF3118683F31188E1
:10A62000FFF7A2FF0546A0B9A368E2689A4218BFE7
:10A630000133A360236943B3042104F11000FFF741
:10A6400089FC10B3FFF760FF3046BDE87040FEF7AD
:10A65000A3BE1030FFF7ACFF2846FFF777FF0023BB
:10A66000EB66EFF305830D2B0FD81BB1084B5B682E
:10A670001B050AD5074B9B685B897F2B05D8FFF725
:10A680008FFE003018BF0120DBE786F3118870BD14
:10A6900000ED00E0A014002038B54FF02003EFF3E8
:10A6A000118483F3118883682BB1013B836084F3A9
:10A6B0001188002038BD21B984F311886FF00F0094
:10A6C00038BDFFF75DFEFFF71FFF2046BDE83840AD
:10A6D000FEF762BE034BD3E900010A23A0FB03018E
:10A6E000704700BFC81600202DE9F34706464FF01B
:10A6F0002003EFF3118083F311885A49D1E9004513
:10A70000A21945EBE673C1E9002380F3118868467E
:10A71000CDF800D0CDF804D04FF02003EFF3118432
:10A7200083F31188504D2A46214652F80C3F93423C
:10A73000944600D0FBB984F31188A868FFF7C0FEE7
:10A74000B0B14A4B1A680A2006FB0020484A18603C
:10A75000126890420CDB00221A604FF02003EFF3E6
:10A76000118483F31188A868FFF75EFE84F31188D3
:10A7700002B0BDE8F0871C693E4FA41B1C61012498
:10A780003C606FF001041A69D2B993E80440CEF836
:10A7900000201A68C2F804E0009A1A60009A586013
:10A7A000009353601C6181F311884FF02003EFF395
:10A7B000118183F31188EB68634501D0002BE2D14E
:10A7C00081F31188009B834202D100233B60B4E7F0
:10A7D000002BFAD0019A934214BF1C6800244FF05A
:10A7E000FF384FF0000993E80600116019684A60CD
:10A7F00098684FF02002EFF3118A82F31188C3F8B2
:10A80000108008B3DB6853B14268036813600368C3
:10A810005A60437AC0F81C9023F002034372437AD3
:10A8200023F0040213F01B0F427202D1036A0133BA
:10A8300012D08AF31188002CC7D0019BA3420ED0FE
:10A84000226823461446CEE78AF311885A69002A03
:10A85000F1D018469047EEE7FFF706FDE9E7002242
:10A86000EFE700BFC8160020A0140020C416002087
:10A87000C4150020C016002008B54FF480624FF0C8
:10A88000FF330349034800F08DF9002008BD00BFE5
:10A89000A4360020D0160020437ADA0604D1006ADC
:10A8A000431C5842584170470020704710B501467C
:10A8B0004FF02003EFF3118483F31188437A23F0E0
:10A8C00004034372FFF7E8FF10B984F3118810BD49
:10A8D0000846FFF7C9FC084B9B685B897F2BF4D8BF
:10A8E000FFF75EFD0028F0D0FFF70EFE2046BDE822
:10A8F0001040FEF751BD00BFA014002003695A1C90
:10A9000011D00A4A126990421FBF01680A699B1858
:10A910000B6190E80C001A60026853604FF0FF333F
:10A920000361002070471846704700BFA014002044
:10A93000F0B54FF02003EFF3118683F31188194A25
:10A9400080610A230931B1FBF3F101310162114643
:10A950000023C36151F80C3F8B4200F1100507D171
:10A960000161136943611D60156186F31188F0BDB3
:10A97000002BF5D0D2F810E0046A1F69BC4208DC55
:10A980005A683C1B1C61426103615A6815605D6036
:10A99000EBE7E41B73450462E2D01B68002BEBD1AC
:10A9A000DEE700BFA0140020EFF305800D2807D8D4
:10A9B00038B1044B586880F40060C0F3C020704781
:10A9C0000120704700ED00E0024B9B68187A00F010
:10A9D00001007047A01400204FF02003EFF3118115
:10A9E00083F31188084AD2F82031834206D19B6D47
:10A9F000C2F8203181F31188704713469A6D904256
:10AA0000FBD1826D9A65F5E7A014002008B50446D5
:10AA1000084611461A46A047FFF7D6FF28B1404026
:10AA200080F311884FF0010002DF024B9868FEF7B7
:10AA300025FF00BFA014002070B586B004460E9E0E
:10AA400004960D9E03960C9E02960B9E0F9D0196FA
:10AA50000A9E0096FEF74EFE2DB92046FFF726FF10
:10AA6000204606B070BD29462046FFF761FFF7E794
:10AA7000036D10B5044603B198472046FFF70CFF5D
:10AA800038B12046FFF716FC637A43F0080363727F
:10AA900010BD637A9B0708D594E80C001A60226801
:10AAA0005360637A23F002036372236A0133EBD0AD
:10AAB00004F11000FFF722FFE6E70000F0B5214F98
:10AAC000214D87B03E46BD4205F1300414D31F4BE3
:10AAD0009A68D37A013BD3724FF02003EFF31185CC
:10AAE00083F31188184CB4421FD385F3118807B043
:10AAF000BDE8F040FFF784BC54F8103C049354F8D0
:10AB0000143C039354F8183C029354F81C3C0193F2
:10AB100054F8203C0093A4F130000FC8FEF7EAFD82
:10AB200054F8303CDD642546CDE7616A4B1C03D008
:10AB3000206819B9FFF7BAFE3034D4E7FFF7F8FE02
:10AB4000FAE700BF1804002018040020A014002019
:10AB50000372427200234FF0FF328172C3720262AD
:10AB6000C36183614362704710B504464FF0FF3103
:10AB70002046FFF72BFB034608334268BFF35B8F89
:10AB800053E8001F21F0010E43E800ECBCF1000F78
:10AB9000F6D1BFF35B8FCB0700D59047FFF76CFC76
:10ABA000E4E70000F0B587B004461F460D461646A0
:10ABB000FFF764FA0020059004900290019003973B
:10ABC0000094044B3246294604F11800FFF734FF85
:0AABD00007B0F0BD69AB000070474C
:08ABDC009056FF7F010000000C
:10ABE4005EAE0000990A000000000000F2AC000014
:10ABF400490C00002CAD0000F9AC0000B50D0000BC
:10AC04000000000003AD00009B0F0000BCAD00007D
:10AC14000AAD00006D1100000000000015AD000039
:10AC24006D110000000000005EAE0000E52700008A
:10AC3400000000005EAE0000A98A000000000000D1
:10AC44005EAE0000E9910000000000005EAE00006E
:10AC540075990000000000005EAE00007D9C0000BD
:10AC6400000000005EAE00006D9F000000000000C8
:10AC74005EAE000015A50000000000005EAE0000FE
:08AC840079A8000000000000A7
:10AC8C0000FFFFFFFFFFFF0011223344556677885A
:10AC9C009900112233445561726763203D2025646D
:10ACAC000A002020617267765B25645D203D2025BB
:10ACBC00730A00706F6E670A0073616D706C655F6C
:10ACCC006D6F64756C650070696E670070617261A0
:10ACDC006D73007072696E742061726763001B5B28
:10ACEC0073001B5B7500554152545F3000737973D0
:10ACFC005F636C6F636B004750494F5F3000636C50
:10AD0C006B5F6B333273726300636C6B5F6D3136E8
:10AD1C00737263001B5B257544001B5B2575430038
:10AD2C00002000400024F400150C0000B50A0000BF
:10AD3C00D50A0000F10A00000B0B0000350B0000D7
:10AD4C005F0B0000730B0000870B0000930B0000DF
:10AD5C00A70B0000BB0B0000CD0B0000D90B0000B3
:10AD6C00ED0B00002B0C0000010C0000050C00008A
:10AD7C0000000000000200000000000000060000BF
:10AD8C0000010000000300000000000000070000AC
:10AD9C0000000000000000000000000000000000A7
:10ADAC00000400000005000000000000000000008E
:10ADBC000000005000000050006000401510000022
:10ADCC00BB0E00009B0E0000DD0E0000210F0000EA
:10ADDC00610F000000000000D11200000000000014
:10ADEC00000000008511000011110000000000009F
:10ADFC0001000202020000005FAE00000000000033
:10AE0C006D290000F52700007072696F2072656370
:10AE1C00762074687265616420737461636B0025BD
:10AE2C007320287265616C2073697A6520257529F9
:10AE3C003A09756E757365642025750975736167BC
:10AE4C0065202575202F2025752028257520252582
:10AE5C00290A00436F6E74726F6C6C6572006B65BF
:10AE6C00726E656C0073686F77206B65726E656CC3
:10AE7C002076657273696F6E00757074696D65000C
:10AE8C0073686F772073797374656D20757074694E
:10AE9C006D6520696E206D696C6C697365636F6E8E
:10AEAC0064730073686F772073797374656D2068B1
:10AEBC0061726477617265206379636C657300738A
:10AECC00686F772072756E6E696E67207461736B34
:10AEDC00730073686F772073797374656D20737466
:10AEEC0061636B730000F401FA00960064004B0080
:10AEFC0032001E0014007368656C6C3E20000A253D
:10AF0C00730A00257300256300556E7265636F67C5
:10AF1C006E697A656420636F6D6D616E640A0055AD
:10AF2C006E7265636F676E697A656420636F6D6DB1
:10AF3C00616E643A2025730A00496C6C6567616C1C
:10AF4C00206D6F64756C652025730A004D6F6475F8
:10AF5C006C65206E616D6520257320697320746F9C
:10AF6C006F206C6F6E672C2064656661756C742045
:10AF7C006973206E6F74206368616E6765640A0084
:10AF8C00496C6C6567616C206D6F64756C65202510
:10AF9C00732C2064656661756C74206973206E6F08
:10AFAC0074206368616E6765640A00546F6F206D6E
:10AFBC00616E7920706172616D65746572732028A1
:10AFCC006D617820257A75290A00496C6C6567617A
:10AFDC006C20706172616D657465720A0068656CD5
:10AFEC00700073656C656374004D697373696E678B
:10AFFC0020706172616D657465720A0054797065B8
:10B00C00202768656C702720666F72206C697374DA
:10B01C00206F6620617661696C61626C6520636F7C
:10B02C006D6D616E64730A0025732025730A0068C8
:10B03C00656C700A00417661696C61626C65206DAB
:10B04C006F64756C65733A0A000A546F2073656CF3
:10B05C006563742061206D6F64756C652C20656E62
:10B06C00746572202773656C656374203C6D6F6426
:10B07C00756C65206E616D653E272E0A00637963E1
:10B08C006C65733A202575206877206379636C654D
:10B09C00730A002A007461736B733A0A00257325D6
:10B0AC00703A2020206F7074696F6E733A2030787C
:10B0BC002578207072696F726974793A2025640A58
:10B0CC0000757074696D653A202575206D730A00E2
:10B0DC005A65706879722076657273696F6E202577
:10B0EC00642E25642E25640A00464C4153485F307B
:10B0FC00005352414D5F3000464143545553455225
:10B10C004346475F30005045524950485F3000502D
:10B11C0050425F30002A2A2A2A2A204255532046C0
:10B12C0041554C54202A2A2A2A2A0A0020205072DF
:10B13C006563697365206461746120627573206551
:10B14C0072726F720A002020496D707265636973A8
:10B15C0065206461746120627573206572726F7210
:10B16C000A002020496E737472756374696F6E20C7
:10B17C00627573206572726F720A00526573657224
:10B18C0076656420457863657074696F6E2028005D
:10B19C0053707572696F757320696E746572727510
:10B1AC007074202849525120002A2A2A2A2A204821
:10B1BC00415244204641554C54202A2A2A2A2A0A14
:10B1CC00002020427573206661756C74206F6E20B0
:10B1DC00766563746F72207461626C652072656150
:10B1EC00640A0020204661756C7420657363616C81
:10B1FC006174696F6E20287365652062656C6F776A
:10B20C00290A002A2A2A2A2A204465627567206D99
:10B21C006F6E69746F7220657863657074696F6E98
:10B22C0020286E6F7420696D706C656D656E746529
:10B23C006429202A2A2A2A2A0A002A2A2A2A2A2087
:10B24C00257320256429202A2A2A2A2A0A0020204C
:10B25C00457865637574696E67207468726561649E
:10B26C002049442028746872656164293A2025704D
:10B27C000A20204661756C74696E6720696E737460
:10B28C0072756374696F6E20616464726573733A6E
:10B29C002020307825780A002A2A2A2A2A204D5084
:10B2AC0055204641554C54202A2A2A2A2A0A002085
:10B2BC0020537461636B696E67206572726F720ADA
:10B2CC00002020556E737461636B696E6720657224
:10B2DC00726F720A002020446174612041636365BF
:10B2EC0073732056696F6C6174696F6E0A0020204D
:10B2FC00416464726573733A20307825780A0020B3
:10B30C0020496E737472756374696F6E2041636348
:10B31C006573732056696F6C6174696F6E0A002ACD
:10B32C002A2A2A2A205553414745204641554C5438
:10B33C00202A2A2A2A2A0A0020204469766973695D
:10B34C006F6E206279207A65726F0A002020556E2C
:10B35C00616C69676E6564206D656D6F72792061D3
:10B36C0063636573730A0020204E6F20636F7072E5
:10B37C006F636573736F7220696E73747275637427
:10B38C00696F6E730A002020496C6C6567616C20D4
:10B39C006C6F6164206F66204558435F524554556D
:10B3AC00524E20696E746F2050430A002020496C65
:10B3BC006C6567616C20757365206F6620746865B9
:10B3CC0020455053520A002020417474656D7074EE
:10B3DC0020746F206578656375746520756E64657F
:10B3EC0066696E656420696E737472756374696FD7
:10B3FC006E0A002A2A2A2A2A20496E76616C696410
:10B40C00204578697420536F6674776172652045A6
:10B41C0072726F7221202A2A2A2A2A0A002A2A2AC0
:10B42C002A204B65726E656C20416C6C6F63617485
:10B43C00696F6E204661696C75726521202A2A2A13
:10B44C002A0A002A2A2A2A2A204B65726E656C2049
:10B45C004F4F505321202A2A2A2A2A0A002A2A2A04
:10B46C002A2A204B65726E656C2050616E696321CF
:10B47C00202A2A2A2A2A0A002A2A2A2A20556E6BCE
:10B48C006E6F776E20466174616C204572726F72BC
:10B49C0020256421202A2A2A2A0A00437572726503
:10B4AC006E7420746872656164204944203D2025C7
:10B4BC00700A4661756C74696E6720696E7374727C
:10B4CC00756374696F6E2061646472657373203D7B
:10B4DC0020307825780A0049535200657373656EE5
:10B4EC007469616C20746872656164004661746192
:10B4FC006C206661756C7420696E20257321205355
:10B50C0070696E6E696E672E2E2E0A00466174612C
:10B51C006C206661756C7420696E2074687265614C
:10B52C0064202570212041626F7274696E672E0A47
:10B53C000000000060030020C0030020C0030020B6
:10B54C00FC03002008040020F5FFFFFFC0130020BF
:10B55C004B65726E656C20737461636B733A0A0091
:10B56C006D61696E20202020200069646C652020AC
:10B57C0020202000696E7465727275707400776F8C
:08B58C00726B717565756500B5
:10B59400D3AC00008105000000000000D8AC00001E
:10B5A4004D050000DFAC00000000000000000000BA
:10B5B4000000000000C201000000000005150000AA
:10B5C4000000000000000000000000000000000077
:10B5D4000000000000000000000000000000000067
:10B5E4000000000000000000000000000000000057
:10B5F4000000000000000000000000000000000047
:10B604000000000000000000000000000000000036
:10B614000000000000000000000000000000000026
:10B6240000000000F51D0000000000000000000004
:10B634000000000000000000000000000000000006
:10B64400B0000020B0000020010000000100000054
:10B6540000000000000000000000000000000000E6
:10B6640000000000000000000000000000000000D6
:10B6740000000000E4000020E400002000000000BE
:10B6840000000000000000000000000000000000B6
:10B694000001002000010020000000000000000064
:10B6A4000000000000000000020002004C0008003E
:10B6B4000000000068230020280100202801002049
:10B6C4000000000000000000000000000000000076
:10B6D400030003004C000400000000003828002090
:10B6E400FFFFFFFFFF1F00001F000000000000001D
:10B6F40000000000B40800205C080020433700006C
:10B7040000000000BC0800205C080020ED370000A9
:10B7140000000000C40800205C080020433700003B
:10B7240000000000CC0800205C080020ED37000079
:10B7340000000000D40800205C080020ED37000061
:10B7440000000000DC0800208808002043370000C7
:10B7540000000000E408002088080020ED37000005
:10B7640000000000EC080020880800204337000097
:10B7740000000000F408002088080020ED370000D5
:10B7840000000000FC08002088080020ED370000BD
:10B7940000000000880D0020010000007552000028
:10B7A40000000000900D002000000000A5520000E1
:10B7B40000000000D00D002000000000A552000091
:10B7C40000000000B80D00200000000041520000FD
:10B7D40000000000E00D00200000000041520000C5
:10B7E40000000000C80D0020000000000000000060
:10B7F40000000000980D002000000000DD5600004D
:10B8040000000000A00D002000000000DD56000034
:10B8140000000000A80D002000000000ED5600000C
:10B8240000000000B00D002000000000ED560000F4
:10B8340000000000D80D002000000000ED560000BC
:10B8440000000000C00D002000000000B9640000EA
:10B85400FFFFFFFF7DAE00008991000071AE000084
:10B8640085AE0000719100008CAE0000C4AE0000F3
:10B8740059910000AFAE0000D8AE0000FD9000006A
:10B88400CBAE0000EAAE0000F1900000DEAE000096
:10B894000000000000000000000000000090D00341
:10B8A400050000001803002000000000F5B00000AF
:10B8B4002400080700000020FDB000001E0008134B
:10B8C4000000001004B10000180010030000004044
:10B8D40012B1000038001003000000E01BB10000AA
:10B8E4001E000403030000000100000047010000E3
:10B8F40044AC000000000000000000005CAC00004C
:10B90400000000000000000068AC0000000000001F
:10B914000000000074AC0000000000000000000003
:10B9240050AC00000000000000000000F0AB00007C
:10B93400000000002400002014AC0000E4AD00006E
:10B944000000000020AC0000F0AD0000000000008A
:10B95400FCAB0000000000000000000008AC000088
:10B96400C8AD00008C04002080AC00000000000082
:10B97400000000002CAC00000000000000000000EB
:10B98400E4AB0000000000000000000038AC000040
:08B994000000000000000000AB
:10B99C00C5AC0000000000206AAE0000C40200200C
:10B9AC00180400201804002000000000FFFFFFFF17
:08B9BC00000000000000000083
:10B9C40030040020300400200000000000000000CB
:08B9D4000F000000000000005C
:10B9DC004804002048040020000000000000000083
:08B9EC00000000000000000053
:040000030000990957
:00000001FF
